:020000040800F2
:1050000068350020D550000839A90008519E0008D5
:105010000000000000000000000000000000000090
:10502000000000000000000000000000C9B90008F6
:1050300000000000000000009DB0000851C1000801
:10504000E7500008E7500008E7500008E750000864
:10505000E750000829680008E75000083968000890
:1050600000000000E7500008E7500008E750000883
:10507000E750000859A10008E7500008E750000871
:10508000E7500008E7500008E75000080000000063
:10509000E7500008E7500008E7500008E750000814
:1050A000E7500008E7500008E750000871CF0008FB
:1050B00081CF000899A20008000000000000000055
:1050C0000348854600F040FD00480047E5EA000837
:1050D000683500200448804704480047FEE7FEE7A3
:1050E000FEE7FEE7FEE7FEE70DC20008C15000083C
:1050F00030B50B46014600202022012409E00D4670
:10510000D5409D4205D31D469540491B25469540F7
:1051100040191546521E002DF1DC30BDF0B51FB40C
:105120000646002082B005464024019100901BE015
:10513000019922460F46304600F0EAFB049A059B8F
:10514000801A994110D310461946224600F0D0FB30
:10515000361A8F410197224601200021009F00F05E
:10516000C7FB38184D4100902046641E0028DFDC44
:10517000019B00982946324607B0F0BD03460B4319
:105180009B0703D009E008C9121F08C0042AFAD2FD
:1051900003E00B780370401C491C521EF9D2704783
:1051A000D2B201E00270401C491EFBD270470022BF
:1051B000F6E710B513460A4604461946FFF7F0FF16
:1051C000204610BD30B505462A460B4610781C789F
:1051D000521C5B1C002801D0A042F7D0002C03D049
:1051E000002802D06D1CEFE7284630BD421C017834
:1051F000401C0029FBD1801A704730B504460020BE
:10520000034600E05B1C934203D2E05CCD5C401B94
:10521000F8D030BD70B5064608F01CFA04680546A3
:105220000A220021304600F097FB2C6070BDF8B5D3
:1052300002464A40D40F42004B0052085B089A4293
:1052400002D20246084611464A0023D0C30D4A0046
:10525000DDB2120EAD1A202D35DA49020126490AB7
:10526000F6058A19002C00D0524220214F1B11460E
:10527000B9402A411018C20D9A4221D0002C17D0F3
:10528000012D08DCDA05801AD20F8019D207DBB2B3
:1052900000F0A2FBF8BDDA05801A012340001B06CE
:1052A000C01880185A428018CA0F1043490007E0FE
:1052B0004908C2071143DA05801A8019400880188E
:1052C00000F082FBF8BD61000122511A001BF7E7D4
:1052D0000122D2075140AAE70122D2075040A6E797
:1052E000024670B54A40D30FDB0740002DD04A007C
:1052F0002AD0010E140E000212020919400A520AA5
:105300008418E50104465443000A120A2E0450434F
:10531000A4194219200CC543AA18120C0125AD038B
:10532000521C521912047F39240400D0521C10431D
:1053300001D44000491EC2B20C06C0092018401C0E
:105340004008802A02D003E0002070BD40084000E1
:10535000002900DA0020184370BD70B502464A40AB
:10536000D50F40004A00ED0740085208002814D02D
:10537000002A12D0C40DD30D41020120C0055202F3
:10538000490A520AE41A091812187D34914201D3CD
:10539000641C00E04900002C01DA002070BD0023ED
:1053A000914201D3891A0343400849000028F7D1EC
:1053B00000290AD0914202D10121C90705E091429A
:1053C00001D2012101E00121C943E005C0184019C3
:1053D00000F0FAFA70BD420005D04200120E5242AF
:1053E0008A4201DB00207047C90508187047000099
:1053F000F0B507460846584087B0C00F04904800F3
:105400000E46590040084908BC1A884105D2384662
:1054100031461E4617460B460246580040081043C8
:105420004CD0300D039040055900400D490D0590BA
:10543000401A0290402872DA18030121000B090576
:105440000843019004980092002805D00199524227
:105450000020884100920190029840210A1A019987
:10546000009800F045FA05460C466B4607CB00F065
:1054700060FAC0197141039A0E0D0023D7175640E8
:105480001A467A40164344D0049A002A2DD0029A34
:10549000012A039A15DC1205C01A9141012636052E
:1054A000001C7141D20F059ED20700930192029613
:1054B0002A46234600F0D6FA07B0F0BD38463146FA
:1054C000FAE71605224A0F46B218C01AB741012161
:1054D0000905001C4F4100187F41114618187941F9
:1054E000E20F10436D19644113E0E2076D081543A4
:1054F0006408C2071443039A01261205C01A914199
:105500003605001C7141CE07400830434908C018D9
:1055100051412A46234600F098FACDE7FFE7049868
:1055200001224000C117121A00238B410498314612
:10553000C417381AA141EEE730B40124E4076340F0
:1055400030BC55E730B40124E407614030BC4FE77C
:105550000000E0FFF0B51FB488B00B990998002453
:1055600048400999C00F490049080991C0070B99A3
:105570000090490049080B9109990898A6460843EC
:105580001CD00B990A98084318D0099801244000B0
:10559000420D4800410D099824050003000B2043EB
:1055A00009900B980003000B20430B9050181C49E6
:1055B0004018002201901446104605E000200146E4
:1055C0000DB0F0BD032801DA034600E003239C463A
:1055D000C11A0AAE0AE05F0008ADED5B4F00F75B51
:1055E0007D430027AA187C41491C5B1E6145F2DD02
:1055F000410004AB5A522104120C0A43240C401CF3
:105600000828DFDB01980290009970460191009014
:10561000059B049A0799069800F024FAD0E7000049
:105620000DFCFFFFF0B50C465C4085B0E40FE407CD
:1056300003944C0000266408590094464908024629
:105640000296224321D062460A431ED06200570DC3
:105650004A000E032303550D012402462C4924055C
:10566000781B1B0B360B40182343264361460090E2
:105670001C46501AB44103D30098401C009002E02D
:10568000921800985B41002803DA0020014605B01B
:10569000F0BD0020012109050746864611E0644659
:1056A0001D46141BB54106D36546521BB3417446D3
:1056B00007430C43A646CD074008490828439218E3
:1056C0005B4105460D43EAD11046184313D06046AE
:1056D000194650407140084306D06046101AB34145
:1056E00006D20122002306E000220123DB0702E0AC
:1056F0000122D2435310009874460105381C6141C1
:10570000029C039D0019694100F09FF9BFE700006A
:10571000FD03000070B54B005B0803430BD04B004A
:105720005C0D002633466542B341D417AD1AA34140
:1057300002DB0020014670BD12053018514170BDDA
:1057400010B500229623114600F046F910BD000066
:105750000EB5C217C10F5040CA0740180021054BB3
:105760000293019200910A460B4600F07BF903B0C8
:1057700000BD0000330400000EB505490291002170
:1057800000910A460B46019100F06CF903B000BD90
:1057900033040000410040020122400AD205090EF4
:1057A00080187F2901DA00207047962903DC9622B1
:1057B000511AC840704796398840704770B5CD0F70
:1057C0004A0009030123090B1B0519430B4BED0785
:1057D0000024520D9A4201DA002070BD074B343389
:1057E0009A4203DC9A1A00F093F802E00449511837
:1057F00088402C43F1D0404270BD0000FF03000000
:10580000CDFBFFFF4A0009030123090B1B051943C8
:10581000094B10B5520D9A4201DA002010BD064B1B
:1058200034339A4203DC9A1A00F072F810BD03492F
:105830005118884010BD0000FF030000CDFBFFFFA2
:10584000C20FD207400040080BD0C10D0723DB0177
:10585000C91840020905400A1143C2084007114314
:10586000704700200146704710B5002904DB012471
:10587000E40740428C412146002B04DB1C460123F7
:10588000DB075242A3418B4200D1824210BD00008F
:1058900010B5002904DB0124E40740428C41214675
:1058A000002B04DB1C460123DB075242A341994233
:1058B00000D1904210BD0000CB0FDB07490010B5AE
:1058C000490802460A4307D00A0D07240903E401E8
:1058D000090B121B002A01DC002010BDC900440F77
:1058E0000C43C100E018D205801800F06DF810BD1F
:1058F00010B5202A04DB0146203A9140002010BD5B
:10590000914020239C1A0346E3401943904010BD68
:1059100010B5202A04DB0846203AD040002110BDF3
:105920000B46D340D0402024A21A91400843194688
:1059300010BD10B5202A06DBCB170846203A1041CF
:10594000C1170B4306E00B461341D0402024A21A96
:1059500091400843194610BDF7B5009C0F4600263C
:105960002578641C002D05D000F000F90068405D2A
:10597000C007F5D12B2D02D02D2D18D0641E39462D
:105980002046029A00F0F6F8002F04D03968A142B0
:1059900001D1009939607105022400290BDA4042D7
:1059A000002803DD07F056FE0460A007FEBD0120BD
:1059B00080020643E3E70028F8DA07F04BFE0460B4
:1059C0000048FEBDFFFFFF7F002904DA401C4900AC
:1059D00001D140084000704770B40024050C05D187
:1059E0001024000402D1002921D01124050E01D178
:1059F00000020834050F01D10001241D850F01D1DB
:105A00008000A41C002801DB4000641C002908D091
:105A100020252E1B0D46F540A14000D00121294331
:105A2000084301061B1B000ADB1D02D5002070BCC9
:105A30007047DB05181880180029F8DA401C490067
:105A4000F5D170BC40084000704710B5002B08DA53
:105A50000024401C614192185B411A4301D1400867
:105A6000400010BDF0B51FB482B005460C0003D055
:105A7000084607F095FD02E007F092FD203002464F
:105A8000009021462846FFF733FF049B059A044601
:105A90000F4618431143084314D0184610431BD037
:105AA000009840210A1A18460599FFF731FF05466C
:105AB0000E46009A05990498FFF71AFF084305D08F
:105AC000012004E02046394607B0F0BD0020C11790
:105AD00005430E432C43374300990E986305401A43
:105AE0007905E40A00220C43FD0A0A3002D50020A1
:105AF0000146E9E70105101969410C9C0D9D00194B
:105B00006941FFF7A2FFDFE74A0009030123090B00
:105B10001B0519430A4B10B5520D9A4202DA0020B8
:105B2000014610BD064B34339A4203DC9A1AFFF744
:105B3000EFFE10BD034BD218FFF7DAFE10BD0000D8
:105B4000FF030000CDFBFFFF064C0125064E05E0DC
:105B5000E36807CC2B430C3C98471034B442F7D38E
:105B6000FFF7B2FA34F2000854F200080048704718
:105B700094F00008F7B582B0029C00272078641CDE
:105B800015460197302802D0002D15D015E0207859
:105B90000127641C782804D0582802D0002D09D091
:105BA0000BE0002D01D0102D07D100271025207803
:105BB000641C02E0082500E00A250026009610E09B
:105BC0000099012769430818020C294680B27143E5
:105BD00000908E183804864201D30120019020786D
:105BE000641C294600F019F80028E9DA0398002817
:105BF00005D0002F01D0641E00E0029C04600198D3
:105C0000002806D007F026FD02210160C81E05B05D
:105C1000F0BD009930040843F9E73A2800D2303843
:105C2000202302469A43412A01D31046373888423E
:105C300001D30020C043704770B58C180578401C14
:105C40006B075B0F01D10378401C2A1106D1027843
:105C5000401C03E006780E70401C491C5B1EF9D105
:105C60002B0705D40023521E0DD40B70491CFAE7F4
:105C70000378401CCB1A921C03E01D780D70491C60
:105C80005B1C521EF9D5A142D8D3002070BD70B55F
:105C9000044620688168490727D58168102549078F
:105CA000002905DA8168890702D481682943816067
:105CB00001F0DAFD064620688068400715D501F03E
:105CC000D3FD801B0A280CD920688068400708D5BE
:105CD000606D28436065A06D01210843A065012027
:105CE00070BD206880684007E9D4002070BD0000C6
:105CF00038B50446094808490068FFF7F9F96043D8
:105D000000900098002805D00098401E0090009850
:105D10000028F9D138BD000040420F00F4010020F6
:105D2000F8B50446206881688907890F012934D1B4
:105D30000168C90731D0816805221140102501266C
:105D4000012907D0606D28436065A06D3043A065D0
:105D50000120F8BD8168022211438160216803207F
:105D6000086001F081FD074620688068C00714D0F4
:105D700001F07AFDC01B0A280BD920688068C00793
:105D800007D0606D28436065A06D3043A065012099
:105D9000F8BD20688068C007EAD10020F8BD000087
:105DA000F8B50446206881688907890F012902D166
:105DB0000168C90733D181681A4A102611400125AC
:105DC000002907D0606D30436065A06D2843A06551
:105DD0000120F8BD8168294381600120FFF788FF19
:105DE00001F042FD074620680068C043C00716D096
:105DF00001F03AFDC01B0A280CD920680068C04396
:105E0000C00707D0606D30436065A06D2843A06572
:105E10000120F8BD20680068C043C007E8D1002019
:105E2000F8BD00001700008010B50E4801F004FB1B
:105E300000F0BAFA05F0C2FF00F0FCFD0A480B4979
:105E4000C08C08600A4C0020A06000F0B1F809483E
:105E500000F058FF00F028F9207004F05DFA0020EF
:105E600010BD0000B80B0000A8070020280000208B
:105E700038000020296A0008F8B503F03BFD04F063
:105E8000EDF800F0E7FE04F089FA3A4D2878002892
:105E900001D108F0DBFD04F069FA0026364C012838
:105EA00010D100F0EDFD01280CD1E078002809D1D7
:105EB000204618308188006801F0C8FC012801D014
:105EC00005F038F92B480125007800283AD12B48F5
:105ED0000078002832D06079294F002804D00128AA
:105EE00018D0022835D125E03868A168411A254824
:105EF000C08C814205D86078012802D0E079012861
:105F000027D1E671667020A003F0BAFB05F0FEF819
:105F100065710CE03868A168401A3C2819D9A57051
:105F2000E5701CA003F0ACFB05F0E4F8667138687E
:105F3000A06007E0A570E57019A0F3E705F0DAF8B6
:105F40006671E5710B480078012802D105F0D2F89E
:105F50006671094810308188006801F077FC0128DB
:105F600004D000F02BF926710020F8BD00F044F9B0
:105F70002571F9E7300000203800002002000020E1
:105F800028000020A8070020475053204F4E0D0A3C
:105F900000000000475053204F46460D0A00000005
:105FA00047505320535543434553530D0A000000B7
:105FB00010B5012008F0FCFD0A4C1328A0700AD08F
:105FC000E01C04F07DF8E078A070332806D0064984
:105FD0000020C88710BD08F023FE10BD04F042F871
:105FE00010BD0000A00100206807002010B500F0DF
:105FF00003F8002010BD000070B50524FF2224071F
:1060000001322146012005F08DF81749002007F0E4
:10601000B3F81649022007F0AFF81549012007F040
:10602000ABF8144D012292032946002004F0A8F990
:1060300004222946012004F0A3F901221203294673
:10604000022004F09DF910222146002000F0FAFD04
:106050000021094800F0F2F80122D2022146012075
:1060600000F070F8002070BDC00500204806002038
:1060700038050020000400502807002010B5002437
:10608000084801F007F9611E064801F09BF8002856
:1060900003D1044800F070FF0446024801F02AF9D9
:1060A000204610BDAC04002070B5002400F026F896
:1060B0000D4E0546B04215DB00200C4A0C4B014644
:1060C000FFF7E6FB01D264240CE031462846FFF7D7
:1060D000FFF80849FFF741F90749FFF701F9FFF712
:1060E00059FB0446204670BD33335340CDCCCCCC55
:1060F000CCCC10406666663F0000C84210B500F088
:1061000017F8642001F098F9FFF7B8FF00F03EF8A7
:10611000044600F003F8204610BD000010B5034807
:1061200001228189806801F098FB10BD681600206B
:1061300010B5034800228189806801F08EFB10BDF4
:1061400068160020022802D30020C0437047C30015
:106150000248C1501818828000207047681600203D
:1061600010B5084C206B00280AD16169A06A401A5A
:106170003C2805D3FFF798FF03490870A06A6061C7
:1061800010BD0000000000203800002010B5FFF70F
:10619000F3FA0022064BFFF745FA064A064BFFF7D3
:1061A000D9F9FFF789FB0121FFF715F910BD0000B0
:1061B00000FEAF406666666666660A4010B50D4C26
:1061C0000023204600686168026800290BD004297A
:1061D0000BD008290BD0136402F054FD206802F0A4
:1061E000C3FB002010BD5363F6E79363F4E7D3636A
:1061F000F2E700004C01002010B50F4C206802F0BF
:1062000083FB03CC083C02F0F3FC61683C200029CE
:1062100008D004290AD00829216809680AD008642E
:10622000002010BD216809684863F9E72168096802
:106230008863F5E7C863F3E74C010020014A03C215
:10624000002070474C010020F0B5444D89B0002477
:10625000434867000246015D5C32D153032909D0EF
:106260003F49A2003F4830398850641C0B2CEFDBBB
:1062700009B0F0BD022101553948A600F830805917
:10628000FFF766FA384A394BFFF764F9FFF714FB5A
:10629000686502903248A96DCC308059401AFFF7EA
:1062A0006BFA69672867059106902D482C49A03044
:1062B000743180598959401AFFF75EFAE967A86777
:1062C000049003917F20C0050299FFF701F8FFF7C2
:1062D000B7FA039B049AFFF73DF9059B069AFFF76F
:1062E00031F90022D243FFF715FA214A214BFFF77B
:1062F00031F91A4A204B803203C213221206FFF7EB
:1063000029F9E96600221D4BA866FFF7C1FA1FD2E2
:1063100000221B4BE96EA86EFFF7A6FA18D21948A7
:10632000C05FFFF715FA039107460022164BE96E8E
:10633000A86EFFF70FF93A46039BFFF759F8FFF7EE
:106340003DFA074930398851E87A401CE8728CE7F9
:10635000034904483039885187E70000A000002035
:106360008C0E0020FFFF0100143BB1133BB103BEB4
:10637000FA48CE3B1835B13D19DDB141000024C0CB
:1063800000408F40B00F00200000594010B500239E
:106390001A4603E0845CE3189BB2521C8A42F9D38C
:1063A000D84380B210BD000000B587B00121684617
:1063B0004170022101700D480190C80102908000D7
:1063C0000490402005906946002006F021FE074811
:1063D0000749203801610749C161074981610749BF
:1063E0004161074803F07CF907B000BD6815002043
:1063F0001164000805640008416400084F64000847
:10640000C80F002010B50146002006F0C1FD10BDE8
:106410000FB400B5FFB082B0012183AB49026846DA
:10642000829A07F0A7F86846FEF7E0FE0246694642
:10643000002006F005FF7FB002B008BC04B018478A
:1064400001B501226946002006F0FAFE08BD10B52C
:106450000446FEF7CBFE02462146002006F0F0FE81
:1064600010BD30B4446C1C252C400125A540046CA3
:106470006560046863608368102B05D003689960C9
:106480000068C26030BC704703689A600068C160F1
:1064900030BC704708B503E06846007806F07EFF20
:1064A0006946002006F074FD0028F5D008BD000004
:1064B000F8B50A2008F077F97D20400108F08EF940
:1064C000A24C00266670A248E0646676607C0C28C8
:1064D00001D30B2060740A2121719E48A6709E4D45
:1064E000007828719D4A6079127840001043A27D9F
:1064F00092001043227E52011043E871E06AE87076
:10650000020A2A72401CE062A974284614229449A7
:106510001330FEF733FE924928462C222730603193
:10652000FEF72CFE8E49284616225330EC31FEF73A
:1065300025FE8C480021415E002903D08A4A128A38
:10654000511801808449027850314A764078887623
:106550001A20687285480078A872A07F28730846C0
:106560007A49633820310A780275497841756D207F
:106570000022794908F002FA20790021C0001D307C
:1065800008F00EFA06F0C6FF022008F05DF90026BA
:10659000EE71A674A67301202074E673744801F0AE
:1065A000BBFAA0840546A6702079FFF7E5F8714A8A
:1065B000714BFEF7CFFF07F089FD00226F4BFEF70E
:1065C00017FFFFF71FF90006C00C401980B2012128
:1065D000C903E084884201D3401AE0846848A0637C
:1065E000E078401CE070624801F096FA6084654EE5
:1065F00053E05F4801F090FA6084634D0AE05C4824
:1066000001F08AFA80B26084E18C884202D3891951
:10661000884206D300210F2008F032F82842206378
:10662000EDD0206B411C22D0400436D58122D2010E
:1066300000210F2008F077F90021102008F020F841
:1066400041064748490E0022A438A16408F068F8C2
:1066500008F02AF82065002008F0C0F8002008F0B3
:1066600078F83F48A438417A172902D008E006F0AC
:10667000D5FF02224549401DFEF7BFFD002833D05B
:106680002A4600210F2008F04EF92079A178401CFD
:10669000814202D0002008F05CF8618CE08C8142DD
:1066A000A7D380198142A4D807F0FCFEFFF7CCFDE8
:1066B0002B4D374900202A4660328300D3588B4245
:1066C00002D219464300EF5A401CC0B20B28F4D343
:1066D00027840020607301202B4A20708032002123
:1066E0000F2008F020F9F8BD08F09CF9E165A065DD
:1066F00008F085F961661A4920660346AB390A7AC3
:1067000068460270497A4170A578018814486A0089
:106710008152134A82380090863A2846111F05F0AC
:10672000B7F90F490320903148550D48A900603052
:1067300040586063A06C2628AFD109496800EC314D
:10674000411807488C3800880880A6E7A000002080
:106750003F420F0038000020A40C00205800002009
:10676000FC0D002082000020A807002070000020FF
:10677000080500209A9999999999E13F00000840ED
:10678000A0860100983A000000D027246000002075
:10679000FFFF01001449012048720A4602205E32C0
:1067A000507203203C3A507204200E3A50720F4847
:1067B0000D4B0078087022310870203108770C49A1
:1067C0005A1C087858714978997123331871597196
:1067D000203318775977107551751A461E32107587
:1067E0005175107651767047300C002066000020FD
:1067F0006000002010B505F0BFF8202005F07AFCFD
:10680000012007F077FE002005F074FC044807F033
:106810000FFD044807F0D8FF002008F00DF810BD68
:106820008C0000208380000010B5012000F048FF9C
:10683000022000F045FF10BD10B5202000F040FF01
:10684000802000F03DFF0120400200F039FF10BD24
:1068500010B4084900234B6107494A684C1522438C
:106860004A604A68082422434A60C009C0010360A4
:1068700010BC7047502E0020002002407FB500253C
:106880000C460646039500F055FEE009029003A968
:1068900001960095684600F0E1FD002804D000F064
:1068A0001DFE002004B070BD00F018FE0120F9E7C5
:1068B00010B5002302E0C45CCC545B1C9342FAD3B5
:1068C00010BD000010B40020204A9169CB0520497A
:1068D00004D54869022318434861901593699B05C4
:1068E00005D54B69012423434B6163021843936927
:1068F0005B0505D54B69082423434B61E30118432D
:1069000093691B0505D54B69042423434B6163023E
:10691000184393699B0405D54B69102423434B61AD
:106920006302184393699B0304D54C6920231C43DD
:106930004C6118439369DB0305D54B69402423431D
:106940004B61A1020843906110BC704700200240D7
:10695000502E002070B5044600F086FF0546194E03
:10696000B069C0070DD0601C08D0002C04D000F026
:106970007BFF401BA04201D9032070BDB069C00756
:10698000F1D1B069800701D50220B061B069C005BE
:1069900011D4B06980050ED4B06940050BD4B0693C
:1069A000000508D4B069800405D4B069800302D41E
:1069B000B069C00303D5FFF785FF012070BD00203B
:1069C00070BD000000200240F8B5174600260546BD
:1069D0000C4600F0AFFD09E029460220226800F0D5
:1069E0008BFD002804D1241D2D1D361DBE42F3D37E
:1069F00000F074FDBE4201D20020F8BD0120F8BDB8
:106A000010B5084902460020054B097905E044000D
:106A10001C5B944203D0401CC0B28842F7D310BD27
:106A2000FC0D0020A00000200149022048717047A1
:106A30003800002000B587B0012069464870022068
:106A400008700C490191410202910B490391052103
:106A5000490204910590694606F0DAFA8821074850
:106A600002F0F2FF052001221021000700F0F5FEE0
:106A700007B000BDF8160020F81A002008250020F5
:106A800003480078002801D000207047012070479B
:106A900058010020F0B593B00E460546282108A8FD
:106AA000FEF785FB03AA00922846314601AB41A2BE
:106AB00002F0FBFF0027FF4302281AD10499039834
:106AC00002F0E3FFC2B201980178012003E0019BCC
:106AD0001B5C5940401C029B8342F8D8914208D16C
:106AE000002406AB36A23146284602F0DEFF0F280E
:106AF00002D0384613B0F0BDA819801E047044704F
:106B00003B482B4602783B4841880492029103940B
:106B1000059439498088097801910090FF2137A2B6
:106B200001313D4803F0B4F8074680213B48FEF7A9
:106B30003EFB3A4638493948FEF720FB384D394E7E
:106B4000AF700698394600783028334824D002F0D8
:106B5000B7FD686800281DD033A002F091FD6B6876
:106B60003A462D4900209847687800281ED0FF201B
:106B700019E0314920460C60304903460C60304929
:106B80000C600146326804F05DFF642000F054FCA4
:106B900004F074FF0020ADE702F092FD6878002851
:106BA00004D0FF20000230606C70E2E70120346006
:106BB0006870DEE72425702A25700D0A00000000A9
:106BC00024252A2C252A2C252A2C252A2C252A2C3A
:106BD000252A2C25702C252A2C252A2C252A2C25E3
:106BE0002A2C252A2C252A2C252A2C252A2A000065
:106BF0003C000020680700203800002025732C2569
:106C0000582C253032782C25782C25642C25782C8E
:106C10002564250D0A00000090250020781600202C
:106C2000580100201C0000204C4F52412046414694
:106C300041464146410D0A0024000020200000206A
:106C400018000020C3000248C15018188280704705
:106C5000F824002008B500206946087003E0684663
:106C6000007800F013F86946022006F091F9002838
:106C7000F5D008BD01490020087070475801002078
:106C800001490120087070475801002070B51A4D65
:106C900000262C462B78611C8034002B08D022461D
:106CA0005268022B0CD0032B09D10A2813D021E003
:106CB000242804D102222A7070540120606070BD23
:106CC00050546168491C61607E2913D20D28F6D1A9
:106CD0000320287070BD50546068401C60604654AA
:106CE00006A1681CFEF76EFA002803D0681C6168D4
:106CF000FFF7D0FE2E7070BD082500204747412CBD
:106D00000000000001494860704700005801002061
:106D100070B50024204604F059F93C493C48A200D3
:106D2000641CE4B281500C2CF9D33B4939480A78F1
:106D300002754978417539490A7802764978417671
:106D400034491520133148720A2007F02CFD7D20AC
:106D5000400107F043FD2F49002213310C2007F0BA
:106D60000DFE00210C2007F01BFE06F0D3FB0220D5
:106D700007F06AFD002004F029F9274C284D203C3B
:106D800000210F2007F07CFC28422063F8D0206B04
:106D9000411C38D0400435D58122D20100210F207A
:106DA00007F0C1FD0021102007F06AFC41061948D8
:106DB000490E0022C73007F0B3FC164DC735687A7C
:106DC00015281FD102221549681DFEF716FA002862
:106DD00018D11148AE7C26710422691C2430FEF7BC
:106DE000CDF929461331084672000D469130FEF761
:106DF000C5F920792946420005484838FEF7BEF912
:106E00000320207070BD06F009FC0000FFFF0100A8
:106E10005C0E0020910C0020C000002060000020CB
:106E200000D02724F8B50C4605464035297C0129B9
:106E30000DD00121297401688A68520709D5416D76
:106E4000202211434165002028740120F8BD022052
:106E5000F8BD194B6268D8054710184E9A4215D0F4
:106E60008A6A23685B035B0B1A438A6221684903C1
:106E700005D5B1680143B1600A20FEF739FF2068EB
:106E8000800315D5B0683843B06011E08A6A236882
:106E90005B035B0B9A438A622168490302D5B168A0
:106EA0008143B1602068800302D5B068B843B06008
:106EB00000202874F8BD00000110000000270140E8
:106EC00070B50446002C0AD0606D0221084360654D
:106ED0002046FEF7DCFE0546280002D009E001202E
:106EE00070BD2046FEF71CFF0546012D01D0012094
:106EF00060650026012D32D0206841681A4A114091
:106F000041602168D043086020688168012212072F
:106F1000914381602068C168144A1140C1602068B3
:106F20000169134A1140016120684169C908C9001B
:106F300041612068016A0F4A114001622068803077
:106F4000416BC909C901416320688030416BC9099F
:106F5000C9014163204600F0F9F8A6656665403432
:106F60002674284670BD000060F7FFFF00023E83D4
:106F700002FCFF3F00F000F00068006C704700006A
:106F800070B50446002C06D0606D264600254036BC
:106F9000002802D006E0012070BDA56535742046AA
:106FA00000F0E8F8606DC00603D4206881684907E6
:106FB00006D5606D1021084360653574012070BDF1
:106FC000616DFF22013291430222114361658168A4
:106FD0005C4A8907890F012902D10168C9072BD1B1
:106FE000032361689B07994205D05B42994202D016
:106FF0005B00994209D10169890089080161206813
:1070000001696368194301610CE00169890089081D
:10701000016190680F2189048843906090686168DD
:10702000084390602068C16818239943C1602068B4
:10703000C168A3681943C16090680121490688436B
:1070400090609068A18E490608439060206881682E
:10705000C90004D4816801221207114381602068AD
:10706000C168394A1140C1602069E268022825D010
:1070700000200243204620300178037B49035B0057
:1070800019430A43216B0A43A16989030A43E16951
:10709000C9030A432168CB681A43CA60616A0A4679
:1070A000FF3AC23A05D0A26A11432268D368194355
:1070B000D16042780121012A02D00BE00420D8E7F8
:1070C0000078002823D0606D202210436065A06DF9
:1070D0000843A065E06B012820D020680169C9073A
:1070E00003D0016949084900016120684169C90864
:1070F000C900416120684169A26B11434161A565E6
:10710000606D80088000401C6065002070BD2068B4
:10711000C26801231B041A43C260DBE720680269CE
:10712000FF239B009A43026120680269236CA66CCE
:107130001A43636C33431A430261206802690A43AD
:107140000261D2E7002701401902FEFF10B5006876
:107150000649884209D10648416B42159143416373
:1071600005200221000700F015FA10BD002401409F
:107170000010024010B586B0044614216846FEF7A0
:1071800016F80E492068884216D10D48416B421509
:1071900011434163C16A01221143C162C06A694659
:1071A00010400590022000900320019000200290E2
:1071B0000520000700F090FA06B010BD0024014041
:1071C00000100240F8B504460E4627466069403775
:1071D00008280BD02068C068C00709D0606D202146
:1071E00008436065002038740120F8BD082500E0E0
:1071F0000C2500F039FB009020680068284219D166
:10720000701C13D0002E05D000F02EFB0099401A00
:10721000B0420BD920680068284207D1606D042174
:1072200008436065002038740320F8BD20680068BA
:107230002842E5D0606D012149020843606520685D
:10724000C16809058A0F0C21002A1BD12022125D7A
:10725000002A17D10268120714D582680123520749
:10726000002A08DB42688A434260606D1A0290433C
:107270001843606506E0606D202210436065A06DD4
:107280001843A065A069002801D120680160002092
:10729000F8BD000070B504460020216889684907E0
:1072A00023D425464035297C01291CD0012129748D
:1072B000E169012902D02046FEF772FD002811D1B4
:1072C000616D0B4A1140FF220132114361650021BB
:1072D000A165297422681C21116021688A68042331
:1072E0001A438A6070BD022070BD022070BD00008C
:1072F000FEF1FFFF70B5044625464035287C012885
:1073000007D001262E742046FEF7C1FC002802D0CB
:107310000CE0022070BD2046FEF702FD002805D1DA
:10732000616DFF220132914331436165002129746F
:1073300070BD30B4014620314A790023022A05D0BD
:107340000422C2630B7130BC0120704702681468CC
:107350000E25AC431460026814686408640014606D
:10736000446C1C22144001252A46006CA240426055
:107370004D710B7130BC1846704770B50024014642
:1073800020314A79022A03D00421C163012418E084
:10739000026813680E25AB431360026813685B082C
:1073A0005B001360436C1C22134001252A469A405F
:1073B000036C5A604D7100220A71816B002900D064
:1073C0008847204670BDF8B504468C460025204607
:1073D00020300179012909D0012606714779002161
:1073E000012F05D0017102252846F8BD0220F8BD05
:1073F00002274771E163206801684908490001607C
:1074000061462046FFF72DF8206B002805D0206844
:1074100001680E221143016009E02068016804221E
:1074200091430160206801680A22114301602068CD
:10743000016831430160D7E770B5044600F014FAE3
:107440000546601C02D004480078241800F00CFAAD
:10745000401BA042FAD370BDE8010020F8B50546F4
:107460000E461B4F387C012808D00120387419487B
:10747000FFF770FA0146080002D025E00220F8BDAF
:107480000020C04330606C68A868C0010019A042A9
:107490001AD92046FFF7DCF90E48FFF75BFA0146E0
:1074A0000D48426808239A434260426843159A4354
:1074B0004260002901D0346006E08034A8686A6820
:1074C000C0018018A042E4D8002038740846F8BDF6
:1074D000502E002050C300000020024005484168A3
:1074E00002221143416041680122114341600020A2
:1074F0007047000000200240F8B50E4617460B4CBE
:10750000207C012808D0012020740948FFF722FAC6
:107510000025002802D006E00220F8BD6561376032
:107520000348FFF717FA2574F8BD0000502E00201D
:1075300050C3000012494868C0070DD0EFF3108017
:1075400072B6104ACA60104ACA6080F31088486850
:10755000C00701D001207047486880070DD5EFF3C0
:10756000108072B6094A0A61094A0A6180F31088DC
:107570004868800701D5012070470020704700004F
:1075800000200240EFCDAB8905040302BFAE9D8C05
:1075900016151413F0B50022002961D00123934081
:1075A0009E460B40002B57D095082E4CAD002D1950
:1075B000AC689607360F0F27B7403C40A446052419
:1075C0002407A04201D1002419E0274CA04201D198
:1075D000012414E0254CA04201D102240FE0244CE8
:1075E000A04201D103240AE0224CA04201D104248C
:1075F00005E0214CA04201D1052400E00624B4405E
:1076000064450FD11D4C26689E43266066689E43E4
:107610006660E6689E43E660A6689E43A660AB6827
:10762000BB43AB60046855000323AB401C430460BC
:10763000D408A4002418266A5507EF0E0F25BD4074
:10764000AE432662C4689C43C46044687546AC433C
:10765000446084689C438460521C0B46D3409DD197
:10766000F0BD000000000140000400500008005080
:10767000000C005000100050001C0050000401409D
:10768000012110B54902202813D0884210D100F002
:10769000CFFF04F063FD03F077F8002005F032FD22
:1076A000012005F02FFD022005F02CFD03F0F8FC71
:1076B00010BD02490020086010BD00002C00002011
:1076C00010B504494A69024202D04861FFF7D8FF69
:1076D00010BD000000040140F0B400220B68002B34
:1076E0006FD001270B6897403B40002B6AD00C7984
:1076F000A407A40F012C01D0022C10D185685400DE
:107700000326A640B543CE68A6402E438660446853
:10771000BC430D79ED06ED0F9540254345600C798E
:10772000E443A40708D0C56854000326A640B54327
:107730008E68A6402E43C6600C79A407A40F022CC5
:107740000CD1D408A40027183D6A5407E40E0F2674
:10775000A640B5430E69A6402E433E62056854001C
:107760000326A640B5430E79B607B60FA6402E43B2
:1077700006604C68A403A40F50D02C4C656B012606
:107780003543656395082A4CAD002F19BD689407F1
:10779000240F0F26A640B54305263607B04201D177
:1077A00000261BE0234EB04201D1012616E0224EF6
:1077B000B04201D1022611E0204EB04203D103268F
:1077C0000CE030E02AE01E4EB04201D1042605E074
:1077D0001C4EB04201D1052600E00626A6402E43ED
:1077E000BE60194DAC689C434E68F60200D51C4340
:1077F000AC60EC689C434E68B60200D51C43EC605C
:107800006C689C434E68B60300D51C436C602C68C2
:107810009C434E68F60300D51C432C60521C0B6839
:10782000D34000D05DE7F0BC70470000001002407C
:10783000000001400004005000080050000C0050FF
:1078400000100050001C0050000401400069084274
:1078500001D00120704700207047002A01D08161CB
:1078600070478162704700000148806870470000DF
:10787000E801002004494A6B01231A434A63034983
:107880004A6802434A60704700100240000001400D
:10789000024881680278891881607047E8010020F9
:1078A00010B50024074801684022114301600320FD
:1078B00000F00AF8002801D0012401E000F080F96E
:1078C000204610BD0020024070B504460E4D7D20BC
:1078D0002978C000FDF70CFC01460C480068FDF754
:1078E00007FC00F061FF002801D0012070BD042CCE
:1078F00007D200222146501E00F08AF96C60002059
:1079000070BD012070BD0000E8010020F4010020DE
:10791000704770470E480F4A816A491C8162C16AEC
:10792000491CC162538F00228B4202D201210163A4
:1079300000E00263084B1878012807D10748016866
:10794000491C0160022901D302601A7070470000CF
:1079500000000020680700203B0000205C000020A1
:107960007047704770472030807B704710B50446E1
:1079700020680168C943C90708D18168C943C9079C
:1079800004D1012141602046FFF7C4FF206801684F
:10799000C943890708D48168C943890704D40221EF
:1079A00041602046FFF7B4FF20680168C9434907DA
:1079B00008D48168C943490704D4042141602046A2
:1079C00000F0FCF820680168C943090708D4816801
:1079D000C943090704D4082141602046FFF7C0FFCE
:1079E00020680168C943C90608D48168C943C9062B
:1079F00004D4102141602046FFF78BFF2068016806
:107A0000C943890608D48168C943890604D4202162
:107A100041602046FFF7A6FF20680168C943490678
:107A200008D48168C943490604D4402141602046F6
:107A3000FFF797FF10BD0000F8B50446002C06D0F4
:107A4000606825462035A87B002802D006E001208A
:107A5000F8BD00206873204600F046F80220A873A5
:107A600020688446C0686168012904D00122A36AA5
:107A7000D205934201D11E229043184B62699A426B
:107A800001D0174B1840174B1840A368676A266A45
:107A90000B433E431E43A36A1E433043002903D1D8
:107AA0002769E6693E433043012903D00121C90516
:107AB0008B4203D12369E1681943084307498A428D
:107AC00005D0A1690A43E1690143104608436146B4
:107AD000C8600120A8730020F8BD0000FFFF00006F
:107AE0003F1FFFFFFEF119FF10B5006808498842EB
:107AF0000CD10848816BC2041143816300221146F6
:107B00000D2000F085F80D2000F076F810BD000083
:107B1000007C0040001002400068C069704700000F
:107B2000F8B50446164602222046203005468273E8
:107B300021480268C3041A4302602068C2689B128D
:107B40001A43C2602068026901273A430261226831
:107B500010205060206881611021204602F07EFBD9
:107B6000032822D021680820486020684661082147
:107B7000204602F073FB032819D0204602F0F4FAE5
:107B80002046FFF7F0FE032813D0206881683943B0
:107B9000816020680169394301612068016904221C
:107BA00011430161AF730020F8BD0320F8BD03202D
:107BB000F8BD0320F8BD000000040140704700003C
:107BC0000448416B012211434163816B020411435C
:107BD0008163704700100240002809DBC106C90E0E
:107BE0000120884003490860BFF34F8FBFF36F8FB8
:107BF0007047000080E100E0002805DBC106C90EE7
:107C000001208840014908607047000000E100E061
:107C10008207D30EFF229A408907090E9940002857
:107C200008DB830809489B001818036893430B433B
:107C3000036070470007000F0838830804489B0062
:107C40001818C36993430B43C361704700E400E015
:107C500000ED00E0024801688215114301607047A1
:107C600000700040F0B4164E326875152A40154B6E
:107C70001B6ADB07DB0F002A04D0002B02D034681C
:107C8000AC4334603468A408A400044334600E4F4D
:107C90003C69042004433C6101290ED040BF20BF51
:107CA00020BF396981433961002A04D0002B02D0FA
:107CB000306828433060F0BC704730BFF1E7000007
:107CC000007000400000014000ED00E0F8B50446FF
:107CD000002620785E4D80067DD55E48806BC00012
:107CE00005D45C48816B02041143816301265A4824
:107CF0000168C90517D40068FF21013108435649BE
:107D00000860FFF7B1FD074653480068C0050AD474
:107D1000FFF7AAFDC01B642801D90320F8BD4E4817
:107D20000068C005F4D54B4F3868032109050840A9
:107D300062681140814208D09003800F032804D16B
:107D40003868800301D50120F8BD286903210904A2
:107D50000840002824D00A40824221D020788006A2
:107D60001ED5286988432A690121C9040A432A616A
:107D70002A698A432A612861C00511D5FFF774FD7D
:107D80000090286980050BD4FFF76EFD0099411A19
:107D90003248814201D90320F8BD28698005F3D516
:107DA0002078800611D560688103890F032905D1E9
:107DB0003A6809058A43084002433A602869032269
:107DC00061681204114008432861012E03D1B96B88
:107DD00030078143B9632078C00705D0E868A168FF
:107DE000800880000843E8602078800705D5E868AF
:107DF0000C218843E1680843E8602078400706D5F5
:107E0000E86803218902884321690843E8602078F3
:107E1000000706D5E8680321090388436169084320
:107E2000E8602088C00506D5E96803200004814386
:107E3000A0690143E9602078000606D5E8680321BF
:107E400089048843E1690843E8600020F8BD000028
:107E500040100240001002400070004088130000F3
:107E6000F8B504460D46002C1BD076480068C007C4
:107E7000C00FA8421CD2734F386840084000284306
:107E80003860FFF7F1FC06463868C007C00FA8420B
:107E90000ED0FFF7E9FC811B6B48814203D9032018
:107EA000F8BD0120F8BD3868C007C00FA842F0D166
:107EB0002078664F800705D5F868F0218843A168CF
:107EC0000843F8602078C00772D06068022808D0A4
:107ED00003280BD001280ED03968890510D4012061
:107EE000F8BD396889030BD40120F8BD39688901D0
:107EF00006D40120F8BD3968490701D40120F8BD36
:107F0000F968890889000143F960FFF7ADFC06466E
:107F1000606802280FD0032820D0012831D0F868EB
:107F20000007800F44D0FFF79FFC811B4648814229
:107F30003AD90320F8BDF8680007800F022837D02F
:107F4000FFF792FC811B4048814201D90320F8BD14
:107F5000F8680007800F0228F2D129E0F8680007CE
:107F6000800F032824D0FFF77FFC811B3648814215
:107F700001D90320F8BDF8680007800F0328F2D16B
:107F800016E0F8680007800F012811D0FFF76CFC9D
:107F9000811B2D48814201D90320F8BDF8680007F4
:107FA000800F0128F2D103E0F8680007800FBAD1F2
:107FB00024480168C907C90FA9421CD90068214992
:107FC0004008400028430860FFF74EFC06461D4865
:107FD0000068C007C00FA8420DD0FFF745FC811B09
:107FE0001948814201D90320F8BD16480068C0072E
:107FF000C00FA842F1D12078400706D5F8680721C4
:1080000009028843E1680843F8602078000707D533
:10801000F8680721C90288432169C9000843F8604C
:1080200000F042F8F9680A4A0906090F515CC84095
:108030000849086008480068FFF746FC0028D3D1CB
:10804000F8BD00000020024088130000001002402C
:10805000F2EF0008F4010020EC0100200148006864
:1080600070470000F401002000B5FFF7F7FF044956
:10807000C968044A4905490F515CC84000BD000069
:10808000001002400BF0000800B5FFF7E7FF0449BD
:10809000C968044A8904490F515CC84000BD00000A
:1080A000001002400BF0000870B5214EF2680C2160
:1080B000104608401F498B0004280CD04D000828AA
:1080C00010D00C2810D070680004410F491C01200A
:1080D000C003884070BD3068C00601D5084670BD39
:1080E000184670BD284670BD9002134C000F205CEE
:1080F0001202940F641CF268D20307D5294605F0DA
:1081000066FA22460023FDF709F870BD3268D206F0
:1081100006D505F05CFA22460023FCF7FFFF70BD90
:10812000194605F054FA22460023FCF7F7FF70BD0C
:108130000010024000093D0002F00008F0B583B0D5
:108140000446002C0FD0F84EF5680C200540F76867
:108150000120000407402078C0075BD0082D09D01B
:108160000C2D03D00FE0012003B0F0BD012000046E
:10817000874208D1306880034CD56068002849D117
:10818000012003B0F0BD012061680004814203D1E9
:1081900031680143316015E0052301221B0492047C
:1081A000994206D131681143316031680143316031
:1081B00008E03168814331603168014001913068E5
:1081C000904330606068002812D0FFF74DFB0290AA
:1081D000306880031ED4FFF747FB0299401A6428D9
:1081E00002D9032003B0F0BD30688003F3D511E05D
:1081F000FFF73AFB0290306880030BD5FFF734FBA2
:108200000299401A642802D9032003B0F0BD3068F7
:108210008003F3D42078800768D5E068810604D510
:10822000326820210A43326088430923042D17D085
:108230000C2D01D1002F13D0002842D03168994372
:1082400001433160FFF710FB0746306840072FD429
:10825000FFF70AFBC01B022827D9032003B0F0BD9B
:108260003168490701D500281CD071681F2212020D
:1082700091432269120211437160316899430143AD
:108280003160FFF711FFF16809060A0FA749895C01
:10829000C840A7490860A7480068FFF715FB0028F9
:1082A000DCD123E0012003B0F0BD30684007CFD51A
:1082B00070681F2109028843216909020843706020
:1082C00014E03068400840003060FFF7CDFA074600
:1082D000306840070AD5FFF7C7FAC01B022802D949
:1082E000032003B0F0BD30684007F4D42078C00606
:1082F0006BD5002D15D0A069002850D03068FF2123
:10830000013108433060FFF7AFFA07463068800557
:1083100036D4FFF7A9FAC01B02282ED9032003B0D8
:10832000F0BD3068800502D5A069002822D07068B1
:10833000072149038843216A084370607068217FE0
:108340000002000A090608437060206A410B491CBC
:108350000120C0038840F16809060A0F7349895C4F
:10836000C8407349086073480068FFF7ADFA0028F9
:10837000D5D12AE0012003B0F0BD30688005C8D512
:108380007068072149038843216A08437060706858
:10839000217F0002000A09060843706015E0316879
:1083A000FF20013081433160FFF75EFA07463068F5
:1083B00080050AD5FFF758FAC01B022802D903200E
:1083C00003B0F0BD30688005F4D420785A4F000720
:1083D0002FD56069002816D038690121084338611B
:1083E000FFF742FA02903869800722D4FFF73CFA7F
:1083F0000299401A022802D9032003B0F0BD38695F
:108400008007F3D515E03869400840003861FFF770
:108410002BFA0290386980070BD5FFF725FA0299ED
:10842000401A022802D9032003B0F0BD3869800742
:10843000F3D42078400775D500200190B06BC000C0
:1084400006D4B06B012109070843B06301200190F5
:108450003A480168C90519D40068FF210131084371
:1084600036490860FFF700FA029034480068C005FA
:108470000CD4FFF7F9F90299401A642802D90320B5
:1084800003B0F0BD2D480068C005F2D5FF20A268FA
:108490000130824203D13969014339611BE0012176
:1084A0008902002A0AD005231B029A420DD13A699B
:1084B0000A433A613969014339610CE03A69824300
:1084C0003A6138698843386105E03A6982433A6124
:1084D000386988433861A068002813D0FFF7C4F9D1
:1084E00002903869800530D4FFF7BEF90299411A2D
:1084F0001348814202D9032003B0F0BD38698005DA
:10850000F2D522E0FFF7B0F90290386980051CD55A
:10851000FFF7AAF90299411A0948814212D90320AA
:1085200003B0F0BD19E0000000100240F2EF0008B7
:10853000F4010020EC0100204010024000700040D7
:108540008813000038698005E2D40198012804D11D
:10855000B06B012109078843B063606A002864D0CA
:108560000C2D49D001252D0602280FD03068A843D4
:108570003060FFF779F904463068800155D5FFF780
:1085800073F9001B022833D90320C9E73068A843D8
:108590003060FFF769F907463068800109D5FFF7B9
:1085A00063F9C01B022801D90320B9E730688001B4
:1085B000F5D4E16AA06AF2680843216BFD231B042D
:1085C0009A4311430843F060306828433060FFF756
:1085D0004BF904463068800127D4FFF745F9001BAA
:1085E000022801D903209BE730688001F5D51CE003
:1085F00030688001C3D418E0012814D0F06801214C
:108600000904A26A014091420BD10F218904E26A58
:108610000140914205D1032189050840216B884220
:1086200003D001207CE701207AE7002078E70000F2
:1086300002480169022211430161704700E000E035
:1086400070B50446002C10D00220254640356874D1
:1086500020680168402291430160204600F064F8E0
:10866000002060656874287470BD012070BDF8B585
:108670000446002C0ED0FF27606A0537002600282C
:108680000AD026616661A66225464035687C0028CE
:1086900007D00AE00120F8BD6068B842F3D0E66177
:1086A000F1E72E74204600F053F802216974206827
:1086B000026840239A4302602123A26860689B02FB
:1086C0001A4038401043E3688A0213401843236974
:1086D0000B40217D1843C907C90F0843A1699310B6
:1086E00019400843E169382319400843216A80236F
:1086F00019400843A16A93001940084321680860A3
:10870000A0690421000C0840616A10231940084345
:10871000216848602068C1699143C1616665012094
:1087200068740020F8BD000010B500680649884252
:1087300009D10648416B8214914341630520E02131
:108740000007FEF727FF10BD003001400010024077
:1087500010B586B0044614216846FCF728FD104980
:108760002068884219D10F48416B8214114341633C
:10877000C16A01221143C162C06A00211040059004
:10878000E0200090022001900320039002910491C8
:10879000052069460007FEF79FFF06B010BD0000E8
:1087A000003001400010024010B40B49401E8842C6
:1087B00002D910BC012070470849486108480723C6
:1087C000C2691202120A4C042243C261002088616D
:1087D0000B6110BC70470000FFFFFF0000E000E0ED
:1087E00004ED00E0024801690222914301617047F3
:1087F00000E000E0F0B402462032137E012B22D0CC
:10880000012616760223537603685D689C687027FC
:10881000BD430F682F435F600068B307984208D0DC
:108820000A4B984205D00A4B984202D0094B984215
:1088300004D180239C4349682143816056760020FF
:108840001076F0BC7047F0BC022070470004004076
:10885000000801400014014010B5022104462034F4
:10886000617601680A6A094B1A4203D10A68520804
:1088700052000A6000F02CF80020A077A076E07685
:10888000207760776076207610BD0000111100001F
:1088900070B50546002D05D02C462034607E00289A
:1088A00002D006E0012070BD00202076284600F0AE
:1088B0001DF802206076291D286803F0AFFC012016
:1088C000A077A076E076207760776076002070BD94
:1088D00000680449884204D10348416B0422914353
:1088E00041637047000801400010024000680449DD
:1088F000884204D10348416B04221143416370470D
:108900000008014000100240014620314A7E012A41
:1089100001D00120704702224A760168CB6801220B
:108920001343CB6000689107884208D00B49884206
:1089300005D00B49884202D00A49884208D1816893
:108940004907490F062906D001681143016002E07A
:1089500001681143016000207047000000040040DE
:1089600000080140001401400168CA685208520022
:10897000CA6001680A6A064B1A4203D10A685208A3
:1089800052000A600121203041760020704700002B
:1089900011110000F8B50446002625462035287E32
:1089A000012817D001202876022068762068826886
:1089B0007727BA43FF231B029A4382600868502836
:1089C00038D00EDC202853D006DC002850D01028E8
:1089D0001ED14DE00220F8BD302849D0402817D1E3
:1089E0003CE0602830D0702819D001221203801A90
:1089F0000FD090420CD1CB684A688968206803F098
:108A00004FFC20688168012292031143816000E0DD
:108A1000012601206876002028763046F8BDCB6814
:108A20004A688968206803F03BFC20688168394304
:108A30008160EEE7CA684968206803F0B6FC5021FF
:108A4000206803F039FCE4E7CA684968206803F04D
:108A5000BEFC6021206803F02FFCDAE7CA68496891
:108A6000206803F0A2FC4021206803F025FCD0E739
:108A700022680146104603F01FFCCAE710B586B015
:108A8000044614216846FCF792FB0D492068884291
:108A900013D10C48C26A02210A43C262C06A019122
:108AA00008400590080300900020029003900620E3
:108AB000049069460448FEF70FFE06B010BD0000A2
:108AC000000801400010024000040050F8B50446C0
:108AD0000D46002726462036307E01280ED0012084
:108AE0003076002A0CD0042A1ED0082A33D00C2A53
:108AF00045D00127002030763846F8BD0220F8BD69
:108B00002946206803F0E0FB2068816908221143B0
:108B100081612068816904229143816120688169B3
:108B2000EA6811438161E5E72946206803F0E5FB27
:108B3000206882690121C9020A4382612068816933
:108B4000012292029143816120688169EA681202E0
:108B500011438161CEE72946206803F0EBFB2068D2
:108B6000C16908221143C1612068C169042291438F
:108B7000C1612068C169EA681143C161BAE7294649
:108B8000206803F0F3FB2068C1690122D20211437F
:108B9000C1612068C269012189028A43C2612068DB
:108BA000C169EA6812021143C161A3E770B50546C5
:108BB000002D05D02C462034607E002802D006E02F
:108BC000012070BD00202076284600F00FF802201A
:108BD0006076291D286803F021FB0120A077A0768C
:108BE000E076207760776076002070BD70470000E7
:108BF00070B505462C462034002908D0042908D039
:108C0000082908D0627F012A07D0012070BDA27E0A
:108C1000F9E7E27EF7E7227FF5E70220002920D07E
:108C2000042920D0082920D060770122286803F089
:108C300029FB0121286889070122884208D00E49B2
:108C4000884205D00D49884202D00D4988420ED194
:108C500081684907490F06290CD00168114301605A
:108C600008E0A076E1E7E076DFE72077DDE701685E
:108C700011430160002070BD000400400008014065
:108C80000014014070B504460D46002229462068B4
:108C900003F0F8FA2068016A0B4A114203D1016817
:108CA00049084900016001202034002D06D0042D20
:108CB00006D0082D06D06077002070BDA076FBE7B7
:108CC000E076F9E72077F7E7111100007047704769
:108CD00070B50446002C1BD02420E0672068016892
:108CE000490849000160206800250560206845604A
:108CF00020688560204600F09BF920468030456062
:108D0000E56705602566656660342576002070BDE0
:108D1000012070BD10B504F045FA10BDF8B5044649
:108D20002268D06911689368A24D06462E40002E35
:108D300009D1850607D58D0605D5A16E002901D07C
:108D400020468847F8BD25468035002E7FD09A4FB3
:108D5000DE07F60F0F40374379D0C70706D0CF059F
:108D600004D5012717626A683A436A60820708D50A
:108D7000DA0706D0276802223A626A6804273A4373
:108D80006A60420708D5DA0706D0236804221A620F
:108D90006A6802231A436A60020709D520220A4042
:108DA000324305D0236808221A626B6813436B6054
:108DB000020509D54A0107D501222368D2021A62A9
:108DC0006A6820231A436A606A68002ABAD080065B
:108DD00006D5880604D5A16E002901D02046884713
:108DE000686821688968490602D42821084228D089
:108DF000204603F0CFFC2068816849061DD5EFF3BB
:108E00001081012282F3108883684022934383609B
:108E100081F31088606F00280BD068498163606F10
:108E2000FEF7ABFA00288DD0606F816B8847F8BDE4
:108E30000DE02046FFF76EFFF8BD2046FFF76AFF02
:108E4000F8BD2046FFF766FF00206860F8BD266E7B
:108E5000012E7DD1C6067BD5CE0679D510231362AF
:108E60002068816826464906403600294CDA626F40
:108E70001168496889B20029E8D0378B8F42E5D95B
:108E8000718311680968890634D4EFF310810122D7
:108E900082F3108802681F01BA43026081F31088D0
:108EA000EFF31081012080F3108820688268520857
:108EB0005200826081F31088EFF31081012080F36B
:108EC0001088206882684027BA43826081F3108846
:108ED0002020286000202066EFF31081012080F31D
:108EE0001088206802689A43026081F31088606FDE
:108EF000FEF71FFA02206066308B718B401A81B238
:108F00002046FFF7E3FEF8BD318B728B891A89B2D8
:108F1000728B002AF7D00029F5D0EFF310820126DA
:108F200086F310880668FF272137BE43066082F368
:108F30001088EFF31082012080F310882068866883
:108F400076087600866082F310882020286000E092
:108F500013E000202066A066EFF31082012080F36A
:108F60001088206805689D43056082F31088022000
:108F700060662046FFF7AAFEF8BDC50208D55B0271
:108F800006D50120000510622046FFF7A0FEF8BDBF
:108F9000020607D50A0605D5E16E0029F7D020465E
:108FA0008847F8BD4006FCD54806FAD5204603F0B0
:108FB00021FCF8BD0F0800002001000425C60008B0
:108FC00010B50446002C03D0E06F002802D007E063
:108FD000012010BD002178200155204600F064F8E2
:108FE0002420E067206801684908490001602046A4
:108FF00003F002FD012819D0606A002802D0204643
:1090000003F042FA206841680922D202914341608C
:10901000206881682A2291438160206801680122CA
:1090200011430160204603F095FA10BD012010BDE8
:1090300010B502681748184982420BD1886B01228B
:10904000920490438863032189021448FEF7A2FA30
:109050001D200EE0124B052000079A420CD14A6BEE
:1090600001239B039A434A6303214902FEF792FAC4
:109070001B20FEF7B1FD10BD0A4B9A42FBD18A6B53
:1090800001235B049A438A630C21FEF783FA1C20B8
:10909000EFE70000004800400010024000040050CC
:1090A0000038014000440040F0B587B00446142168
:1090B0006846FCF77CF8314A2668002530480221D2
:1090C00003230424964218D1826B4E0432438263F8
:1090D000C26A0A43C262C06A6A46084005909802A2
:1090E00023C218C269462748FEF7F6FA0022114645
:1090F0001D20FEF78DFD1D201CE0234F0122BE42E6
:109100001CD1456B960335434563C56A1543C5625B
:10911000C06A6D4610400590032040021FC505201F
:1091200069460007FEF7D8FA002211461B20FEF719
:109130006FFD1B20FEF760FD07B0F0BD134FBE4270
:10914000FAD1866B01277F043E438663C66A1643C5
:10915000C662C06A6E46C007C00F05900C2023C6C9
:10916000052018C669460007FEF7B6FA0022114628
:109170001C20FEF74DFD1C20DCE7000000480040ED
:10918000001002400004005000380140004400403C
:1091900070B580231B58202B01D0022070BD002900
:1091A0000AD0002A08D0012483682403A34209D1ED
:1091B0000369002B02D005E0012070BDCB0701D070
:1091C000012070BD002303660A4C0368A3420ED041
:1091D0005C6824020BD5EFF31084012585F3108819
:1091E0001D680126B60635431D6084F3108803F020
:1091F0003DFD70BD0048004070B580231B58202BFA
:1092000001D0022070BD00290AD0002A08D0012414
:1092100083682403A34209D10369002B02D005E02F
:10922000012070BDCB0701D0012070BD0023036673
:109230000A4C0368A3420ED05C6824020BD5EFF3FE
:109240001084012585F310881D680126B606354374
:109250001D6084F3108803F061FD70BD004800407C
:1092600010B503F0C1FF10BD7047FFB583B00446D1
:109270000F461546E06F202802D0022007B0F0BD4F
:10928000002F0AD0002D08D00120A16800038142E0
:109290000BD12069002803D007E0012007B0F0BD02
:1092A000F80702D0012007B0F0BD00218420015151
:1092B0002120E067FEF7D8FA029026464036358234
:1092C00075820120A1680003814202D12069002833
:1092D00013D03D460027708A00281CD006980090C5
:1092E000002280212046029B03F0E8FD002806D0E2
:1092F0002020E067032007B0F0BD0025EBE7002D3C
:1093000018D02168287888626D1C708A401E70828F
:10931000708A0028E2D10698009000224021204661
:10932000029B03F0CBFD00280BD02020E067032038
:1093300007B0F0BD38882168C005C00D8862BF1C29
:10934000E3E72020E067002007B0F0BD70B50446D9
:10935000E06F202801D0022070BD00290AD0002A29
:1093600008D00123A0681B03984209D12069002876
:1093700002D005E0012070BDC80701D0012070BDFA
:10938000E16420464030028242820021403005469E
:1093900041602120E067206F00281AD0154BC3627E
:1093A000236F15481863236F14485863206F816337
:1093B000206813462830266F02463046E16CFEF7DF
:1093C00002F8002805D0102068602020E067012006
:1093D00070BD216840200862EFF31081012080F306
:1093E00010882068826880231A43826081F3108885
:1093F000002070BD3FC700088BC7000839C60008B1
:1094000030B4C36F202B02D030BC0220704700293B
:109410000AD0002A08D0012483682403A3420BD178
:109420000569002D03D007E030BC01207047CD074F
:1094300002D030BC01207047C164014640310A822D
:109440004A820021C166842211502121C167A342B2
:1094500002D10169002910D00949C166EFF31081DA
:10946000012282F310880068026880231A43026098
:1094700081F3108830BC002070470249C166EDE7D7
:109480005FCE0008FDCD000810B503F045FF10BD0C
:10949000704700000020014908707047A0040020B8
:1094A0000120014908707047A004002070B50446EF
:1094B0000D46204600F02CF8012801D1801E70BD19
:1094C0002268501CE168FBF713FE216023692168C4
:1094D0005943A368C81829462269FBF74FFE0020AC
:1094E000EDE710B58160C26003610124446000248F
:1094F000046010BD10B504462268501CE168FBF7FB
:10950000F7FD6068814201D1012010BD0020FCE719
:1095100010B504462268901CE168FBF7E9FD60681D
:10952000814201D1012010BD0020FCE770B5044646
:109530000D462046FFF7DEFF012801D1801E70BDD9
:10954000236960685843A368C11828462269FBF75D
:1095500015FE6268501CE168FBF7CAFD61600020DF
:10956000EDE770B504460D46002C01D1401E70BDDC
:1095700000BF2068A842FCD32068401B20606268BE
:109580005019E168FBF7B4FD61600020EFE770B5AA
:1095900004460D46002C01D1401E70BD20684019C4
:1095A000206000BFE16820688842FBD8A26850199B
:1095B000E168FBF79DFDA1600020EEE7FFB581B0FB
:1095C00004460D4616460027002E06D004980028B3
:1095D00003D0E1682068884203D30020C04305B06F
:1095E000F0BD2168E068401AA84202D20020C043C2
:1095F000F5E7A0684019E16888420BD9A168E068E6
:10960000471A2168E068401AE919884202D200200E
:10961000C043E4E7A268D019E168FBF769FD316057
:109620007919049801600020D9E70146486870471D
:109630000146886870470246002A01D1401E7047E3
:109640000020506090601060D16000BFF7E70146D5
:10965000002901D1012070470868002801D10120AC
:10966000F9E70020F7E70146002901D10120704702
:109670000A68C868904201D10120F8E70020F6E7A7
:109680000FB400B50D48FFB0007882B0012805D0B6
:1096900000207FB002B008BC04B01847012183ABA2
:1096A00049026846829A03F065FF6846FBF79EFD13
:1096B00002466946002003F0C3FDEAE7540100209A
:1096C00010B5064A1278012A01D0002010BD0A46C2
:1096D0000146002003F0B4FD10BD0000540100203D
:1096E00003490968016002218171014908607047DE
:1096F0001002002000BFEFF30580002800D0704763
:1097000007480068002804D1012080F3108800BFBA
:1097100000BF03480068401C0149086000BFEEE735
:10972000F801002070B504460D4600F04FF80028FF
:109730000FD000F04BF80B21C90140180069002838
:1097400007D000F043F80B22D2018018016902A073
:109750008847002070BD00001B5B481B5B4A00006F
:1097600070B502460C4600210023002A01D0002CCF
:1097700002D10020C04370BD0021002316E0C800C4
:109780000D4D2858002810D1D8001058CD000A4E91
:109790007051D80080184068CD00AD196860074846
:1097A0000068401C054D28605B1C491C502901D2F3
:1097B000A342E4D30020DEE71C02002018020020B0
:1097C0000148006870470000180200200148006846
:1097D0007047000014020020F8B506460F46002529
:1097E00036E0002418E0FFF7F1FF002813D0FFF760
:1097F000EDFF0B21C9014018006900280BD0FFF7CD
:10980000E5FF0B23DB01C01802692819C000134BC8
:10981000195813A09047641C052C04DAFFF7D0FFF9
:1098200029198842DFD8FFF7D1FF00280FD0FFF7B2
:10983000CDFF0B21C90140180069002807D0FFF7B0
:10984000C5FF0B22D2018018016907A088476D1D52
:10985000FFF7B6FFA842C4D80020F8BD1C020020C4
:10986000252D3136730000000D0A00000146202925
:1098700002D30020C0437047012218204843044B04
:109880001A50002218204843C01882600020F2E7D6
:10989000682E002070B505460024002D01D1401E21
:1098A00070BD00240CE0182060430C4908580028C3
:1098B00005D1012118206043084A115002E0641CC0
:1098C000202CF0D300BF202C05D105A0FFF7D8FE37
:1098D0000020C043E4E72C600020E1E7682E002070
:1098E00074696D65722049442069732066756C6CDB
:1098F0000D0A000010B5002400BF41E018206043AD
:109900002149085802283AD118206043401880683D
:109910001E490968091A182060431B4A8018C0684C
:1099200081422CD918206043114640184069002814
:1099300020D01820604340180079002804D101216C
:109940001820604311500AE00221182060430E4A9B
:1099500011500E4801681820604380188160182259
:109960006243094BD218106918226243D218516918
:10997000884704E0012118206043034A1150641C09
:10998000202CBBD310BD0000682E00200002002058
:10999000F0B50446059D202C02D30020C043F0BD45
:1099A0000226182060430E4F3E50182060433E466A
:1099B000801901710B48066818206043C019866041
:1099C000182060433E468019C26018206043801909
:1099D000436118206043801905610020DFE7000023
:1099E000682E00200002002007480068401C06493D
:1099F00008600648026840680021521C484103493B
:109A00000A60486070470000000200200802002041
:109A100000BFEFF30580002800D0704709480068B8
:109A2000002804D007480068401E06490860054821
:109A30000068002804D100BF80F3108800BF00BF79
:109A400000BFEAE7F801002070B504460D4629463C
:109A50002046FBF7ACFB70BD0146302904DB3929F9
:109A600002DC084630380EE0412904DB462902DCDE
:109A70000846373807E0612904DB662902DC08461E
:109A8000573800E00020C0B2704710B502460B46C0
:109A9000002406E01078FFF7DFFF21014418521C74
:109AA0005B1E002BF6D1204610BD0FB4F0B585B07B
:109AB0000446002004900022202003900020029001
:109AC000002C02D00C98002805D1002005B0F0BC75
:109AD00008BC04B018470DA80490CFE0002908D1B5
:109AE0000C980078252803D10C984078652800D080
:109AF000C9E00C98007825286ED10C98401C0C9079
:109B00000C98007803900C98401C0C9003986528E2
:109B100077D004DC2A2807D0642873D113E070289A
:109B200072D07828F9D13EE008E020780C9B1B78B1
:109B3000984202D0641C491E00E001E00029F4D1E3
:109B400000BF521C88E000260196009600230025E5
:109B50002020049E20CE049618E02078009E002E3F
:109B600005D12D2803D10126019600960CE030285E
:109B700009DB392807DC012600960A265E430746E2
:109B8000303FF31900E003E0641C491E0029E4D1D2
:109B900000BF019E012E01D1DE43731C002D00D0B9
:109BA0002B60521C58E000230025049E20CE049612
:109BB0001FE02078302806DB392804DC1E01074628
:109BC000303FF31913E0612807DB662805DC1F012D
:109BD0000646573EBB190AE043E0412806DB46280B
:109BE00004DC1F010646373EBB1900E003E0641C9D
:109BF000491E0029DDD100BF002D00D02B60521C72
:109C00002AE01BE024E0FFE7049E01CE0496002535
:109C10000023254609E026780C9F3F78BE4201D0FC
:109C20005B1C00E003E0641C491E0029F3D100BF67
:109C3000002801D005604360521C0DE0049B01CB5D
:109C40000493002800D00460521C0123029303E017
:109C500001200290002200BF00BF029801280DD110
:109C600011E020780C9B1B78984205D1641C0C985D
:109C7000401C0C90491E01E0002204E00C98007882
:109C8000002800D02AE700BF0020049010461DE7FE
:109C90000FB4F8B506460C46002509A800902146E9
:109CA0003046009B089A03F065FC054600200090B2
:109CB000A54200D3651E2846F8BC08BC04B018476E
:109CC000FEB504460F461546002600200190009080
:109CD000002C01D0002D01D10020FEBD2846FBF74D
:109CE00085FA00900098874201D20020F5E700989D
:109CF000381A0190002609E0A0192946009AFBF7BE
:109D00007CFA002801D1A019E7E7761C0198864269
:109D1000F2D30020E1E770B504460D46002C01D0D7
:109D2000002D02D10020C04370BD0121204610301B
:109D3000FFF717FC20462030A968FFF712FC00202F
:109D4000F2E770B504460D46002C01D0002D02D17B
:109D50000020C04370BD012120461030FFF717FCE2
:109D600020462030A968FFF712FC0020F2E710B56A
:109D70000446002C00D110BD20461030FFF767FCD0
:109D8000012801D10020F6E720462030FFF75FFCD4
:109D9000012801D10020EEE720461030FFF745FCF6
:109DA0000C21484321684018E5E77CB504460E467F
:109DB0000025002001900090002C00D17CBD2046A1
:109DC0001030FFF750FC002801D00020F6E76B466A
:109DD00001AA314620462030FFF7F0FB002801D0D1
:109DE0000020EBE720461030FFF722FC0C2148430F
:109DF00021684518A0680199401828606E60009895
:109E0000A8602846DAE7FFB581B004460E461D4635
:109E100000270C2068430399884202D3781E05B0BE
:109E2000F0BD0C202F4647432660676060688019AC
:109E3000A0600398C11BE160294620461030FFF75F
:109E4000FAFB20462030E168FFF7F5FB0020E6E74B
:109E5000FEE7000010B50E4C002208212046FDF759
:109E6000FCFC002210212046FDF7F7FC0A2004F03C
:109E700098F9012208212046FDF7EFFC0A2004F0A2
:109E800090F9002208212046FDF7E7FC10BD0000F4
:109E90000004005010B50E4C002208212046FDF7AA
:109EA000DCFC012210212046FDF7D7FC0A2004F03B
:109EB00078F9012208212046FDF7CFFC0A2004F0A2
:109EC00070F9002208212046FDF7C7FC10BD0000F4
:109ED00000040050F8B50024144E07462546002221
:109EE00008213046FDF7B9FC0A2004F05AF9012296
:109EF00008213046FDF7B1FC6006040E1021304603
:109F0000FDF7A4FC002801D0641CE4B2052004F095
:109F100048F96D1CEDB2082DE1D3002F03D0FFF7F7
:109F200099FF2046F8BDFFF7B5FFFAE7000400509F
:109F300070B5154E0546002208213046FDF78DFC10
:109F40000024E80901D0012200E00022102130465F
:109F5000FDF783FC6806050E0A2004F022F90122B1
:109F600008213046FDF779FC0A2004F01AF9002296
:109F700008213046FDF771FC0A2004F012F9641C38
:109F8000E4B2082CDDD370BD0004005010B50C4CB9
:109F9000012210212046FDF760FC01220821204605
:109FA000FDF75BFC002210212046FDF756FC0A203D
:109FB00004F0F7F8002208212046FDF74EFC10BD02
:109FC0000004005010B50E4C002208212046FDF779
:109FD00044FC002210212046FDF73FFC0A2004F03B
:109FE000E0F8012208212046FDF737FC012210216C
:109FF0002046FDF732FC0A2004F0D3F810BD000023
:10A000000004005070B5144D002401221021284690
:10A01000FDF723FC062004F0C4F80122082128469D
:10A02000FDF71BFC062004F0BCF807E0641CE4B25A
:10A03000FA2C03D9FFF7C6FF012070BD1021284676
:10A04000FDF704FC0028F1D1002208212846FDF785
:10A0500004FC002070BD00000004005010B5FCF7A7
:10A0600019FA10BD10B53721202000F070F8032137
:10A07000212000F06CF84021222000F068F808212F
:10A08000232000F064F8AA21302000F060F80A488C
:10A0900002210187322000F05AF80121332000F01C
:10A0A00056F85F21202000F052F8044800F008F82C
:10A0B0000A2004F076F810BD68070020A3010020F4
:10A0C00010B501460F2000F021F8002800D0012033
:10A0D00010BD10B50446FFF759FF3220FFF728FFE7
:10A0E000FFF790FFE0B2FFF723FFFFF78BFFFFF7CB
:10A0F0004DFF3320FFF71CFFFFF784FF0020FFF721
:10A10000E9FE0446FFF75EFF204610BD10B50C4681
:10A11000FFF7DFFF2070012010BD70B50D4604462B
:10A12000FFF734FF3220FFF703FFFFF76BFFE0B2CA
:10A13000FFF7FEFEFFF766FF2846FFF7F9FEFFF781
:10A1400061FFFFF73FFF0A2004F02BF870BD10B548
:10A15000FFF7E3FF012010BD10B50248FDF706FC34
:10A1600010BD000008050020F0B583B004460026AD
:10A17000EFF310800090012080F31088344B2068AA
:10A18000C21804D13349CE68032189040E40816886
:10A190000291C168019141698569002A07D12E4861
:10A1A000826AC7043A438262826ABA43826208467C
:10A1B00028433CD026482268C24205D12548C368BE
:10A1C000032292049343C36027462037002910D00E
:10A1D0002068026901231A43026120684161082155
:10A1E000204600F03BF8032800D1B873216808200E
:10A1F0004860002D10D020680169012211430161DF
:10A20000206885611021204600F028F8032800D13D
:10A21000B8732168102048600D482168C14206D1FA
:10A220000C48C1680322920491433143C160206805
:10A230000169490849000161216802988860216824
:10A240000198C860009880F3108803B0F0BD00004A
:10A250000084FFBF401002400010024070B5064667
:10A260000D4600240B480A490068FAF741FF7D219A
:10A27000C90048433268401E002800D103241368F7
:10A280002946994301D00028F5D1204670BD000031
:10A29000204E0000F401002010B50248FEF73EFDFC
:10A2A00010BD00003805002010B5032000F002F8B2
:10A2B00010BD000070B5164D00262C460C3C002841
:10A2C00011D021468978032814D001280AD1491CCD
:10A2D000C8B2A0700C2817D204280FD080002858CC
:10A2E00000F024F970BD00F077F90520FDF7A4F81F
:10A2F000A67001E00029F5D12868F1E70549286931
:10A30000096800F013F970BD00F05CF970BD000041
:10A310006C0100206000002000B587B00120694674
:10A320004870022008700E490191410202910D49C6
:10A3300003918021049105906946012002F068FE96
:10A340000948FFF7A7FA00F047F900F0DFF86420AA
:10A35000FDF772F80020FFF7ADFF002007B000BD49
:10A36000B8270020B82B0020640100200348807823
:10A370000C2801D0002070470120704760010020A8
:10A38000032802D30020C0437047C3000248C150D5
:10A390001818828000207047A0270020FEB50025F5
:10A3A00068460570FF2785802D4C2E4E013734E01E
:10A3B0006846007800F05EF86846027830782254EB
:10A3C000401CC0B2307020182038C17FAA2907D1A4
:10A3D000807F552804D139462148FAF7E8FE3570C8
:10A3E0001F486946408888801F490968884214D1FF
:10A3F000207901280CD1607900280ED1A07901289C
:10A400000BD139461648FAF7D2FE18483570057058
:10A410002079022808D0032810D06946012002F0D4
:10A42000B7FD0028C4D0FEBD0D4968464A790271C7
:10A430008979417181880E48C18409E008496846DC
:10A440004A79027189794171094980884039488780
:10A4500004F0FEFC642003F09DFE03F0EDF8000024
:10A46000A026002060010020600000203A000020AB
:10A47000A807002070B51E491E4B4A78012A05D155
:10A480008A687F2A02D29854521C8A6000220A28C5
:10A4900002D00D2804D029E001208A60487025E010
:10A4A0004A708C68002C21D018192038C277114DC1
:10A4B0004868FFF7DBF910A221462846FFF700FCA9
:10A4C000002805D029460DA0FFF7DAF801200BE09F
:10A4D0000CA221462846FFF7F3FB002806D02946A8
:10A4E00006A0FFF7CDF80220FFF7E4FE002070BDC4
:10A4F00060010020382C00206F6B00005B525D2053
:10A5000025730A006572726F7200000010B503486F
:10A51000012281880068FDF7A0F910BDA027002066
:10A5200010B50020FFF7C6FE10BD00000FB430B517
:10A5300091B015AB402101A8149A03F01BF8002537
:10A5400001A8FAF753FE024601A9012002F078FEA5
:10A5500004460A487D220095074B120100214068FD
:10A56000FFF716FA01A906A0FFF78AF8204611B0F6
:10A5700030BC08BC04B01847A9A200086001002044
:10A580005B535D2025730A0070B505460C480C46E8
:10A5900080780C2802D00020C04370BD00F01CF869
:10A5A0000520FCF749FF22462946012002F048FE1B
:10A5B0000520FCF741FF00F005F8002070BD000009
:10A5C0006001002010B50348002281898068FDF7F2
:10A5D00044F910BDA027002010B50348012281894D
:10A5E0008068FDF73AF910BDA02700201CB50021B6
:10A5F00018480091164A01910260C1631205426039
:10A60000816007228263012202610246C16020321A
:10A610001170FF235170C233436281621173016371
:10A620008161042241634261C161FCF7A9FC0028F9
:10A6300001D072B6FEE70848009080130190694689
:10A640000448FCF7EFFB002801D072B6FEE71CBD02
:10A6500000240140AC04002002000004F0B587B0E3
:10A6600014216846FAF7A3FD4148C26A04210A434F
:10A67000C262C26A0A400592C16A01252943C162C9
:10A68000C16A29400591C26A02210A43C262C06AB6
:10A69000052708403F070590002236493846FDF758
:10A6A000DCF8002234493548FDF7D7F801221103C0
:10A6B0003846FDF7D2F8012240213048FDF7CDF8A9
:10A6C0001126360400246946384601960095029406
:10A6D000FDF702F82A480090029469460195039418
:10A6E0003846FCF7F9FF2448029418380090694670
:10A6F000019503942148FCF7EFFF2248009069463A
:10A70000019602941D48FCF7E7FF09200003009022
:10A710000194694602941948FCF7DEFF1820009066
:10A72000112001900294694603941448FCF7D4FF69
:10A7300040200090032003900195029469460F4841
:10A74000FCF7CAFF2802FDF795F800221146052004
:10A75000FDF75EFA0520FDF74FFA002211460720AB
:10A76000FDF756FA0720FDF747FA07B0F0BD0000E5
:10A7700000100240108900001D410000000400503C
:10A7800010990000A202000010B5FFF72FFF00F0A3
:10A7900009F800F099F800F0B3F800F01FF800F0A5
:10A7A00043F810BD10B50C480A490160E121490287
:10A7B000416000218160C160016181610C22016200
:10A7C00042614162FEF7FCFB002801D072B6FEE751
:10A7D00010BD0000004800403805002010B5114CA5
:10A7E0000F482060FF20053060600020A060E0601E
:10A7F00020616061E0610121206249026062A16123
:10A80000A0620720E0622046FDF731FF002801D05A
:10A8100072B6FEE72068016840221143016010BD56
:10A8200000300140D006002010B58AB00024049406
:10A83000059406940794089422480994009401947E
:10A8400002941F49039401601F21846041600461E8
:10A85000F9214461C160FEF71BF8002801D072B6EF
:10A86000FEE701200003049004A91648FEF792F8C1
:10A87000002801D072B6FEE71248FEF797F90028CB
:10A8800001D072B6FEE7089408A90E480994FDF7B6
:10A89000B1FF002801D072B6FEE76020009001945D
:10A8A00002940022694603940648FEF70FF9002837
:10A8B00001D072B6FEE70348FEF7E0F80AB010BD1B
:10A8C000000801402807002010B50C480A49016023
:10A8D000E1214902416000218160C1600161816123
:10A8E000C1610C22016242614162FEF769FB0028EE
:10A8F00001D072B6FEE710BD00380140C00500204F
:10A9000010B50C480A4901604B21C9014160002182
:10A910008160C16001618161C1610C22016242619B
:10A920004162FEF74DFB002801D072B6FEE710BD74
:10A930000044004048060020FEE70000F0B58BB060
:10A940000A2003F030FF7D20400103F047FFF84C60
:10A9500000256570F748E064607C0C2801D30B206B
:10A96000607420790A2801D90A202071A570207D01
:10A970000127002803D0032801D0277600E02576A0
:10A98000ED48EE4E00783071ED480078F071E06AE5
:10A99000F070010A3172401CE0622079B07442000C
:10A9A0003046E8491330FAF7E9FB2079E54982009F
:10A9B0004000801960311330121DFAF7DFFB207957
:10A9C000062142004843DF498019EC311730921CC0
:10A9D000FAF7D4FBDC490020085E002803D0DB4AEC
:10A9E000128A101808802079D44EC00082190B7882
:10A9F00053764978917616217172D549CC4A0978F7
:10AA0000B172A17F317331462032133913780B753F
:10AA100052784A75002213311D3003F0AFFF2079C0
:10AA20000021C0001D3003F0BBFF02F073FD0220C7
:10AA300003F00AFFF571A574A57301202074E57376
:10AA4000C448FDF769F8A0840646A5702079FAF796
:10AA500093FEC14AC14BFAF77DFD03F037FB00229C
:10AA6000BF4BFAF7C5FCFAF7CDFE0006C10C8819FA
:10AA700080B20121C903E084884201D3401AE084F6
:10AA8000B848A063E078401CE070B248FDF744F895
:10AA9000AC4E6084A43E304622300890001F0290E5
:10AAA000001F0190801E07903CE1AA48FDF734F892
:10AAB0006084AD4F0BE0A748FDF72EF880B26084AC
:10AAC000E18C884203D3A94A8918884206D3002121
:10AAD0000F2003F0D5FD38422063ECD0206B411CE1
:10AAE00021D040047ED58122D20100210F2003F025
:10AAF0001AFF0021102003F0C3FD41069148490EC2
:10AB000027460022A438A16403F00AFE03F0CCFD1E
:10AB10003865002003F062FE002003F01AFE717A0F
:10AB20001729C1D101E002F079FD02229049701D80
:10AB3000FAF763FB0028B7D103F074FFF965B86535
:10AB400003F05DFF79663866B8786A46401CB870D5
:10AB50007C48AB38017A1170407A507010880990A7
:10AB6000398C88427ED1774903209031087008984B
:10AB70000090236E0020029A019900F089FF6F482F
:10AB80007C4F8C30C08E38806C488C30008FA08316
:10AB90007048FCF7C1FF608403F084FCF07C00097E
:10ABA000607513D002227249701DFAF726FB002847
:10ABB0000CD101206149A074C871A06CCA3116384B
:10ABC000C2B26048E2749C30FAF7D8FA6A4805705D
:10ABD0005C48603000686063A063E063F17C090753
:10ABE000090F00E091E0032900D02175A16C26290E
:10ABF00017D152494E4A8C31C98F1185514B079A52
:10AC0000B43312881A8788420ADD002808DD00293B
:10AC100006D0E07D411CE175052802D9257000E0D1
:10AC2000E575E5700120A073E073A08B5349FF30F8
:10AC3000C33080B2A08388420BD949424018A08318
:10AC400038887D21401C80B2C9003880884200D3FA
:10AC50003D8038887D21C9004843A18B401820647D
:10AC6000217900E002E000F03DFF8DE0FBF7C8FE37
:10AC700004900898009004983B6E401CC0B2029A61
:10AC8000019900F005FF2F4A049890320321101813
:10AC90004170049881001046303808184068786385
:10ACA000B86C8C46262807D10498114640005C31C8
:10ACB0004118079800884880224960463031401882
:10ACC000FC39898F01801D4861460B180022796E7E
:10ACD000386E3C46163398540F06000A3843090A6A
:10ACE000521C042AF7DBE26C616B91421ADA154AB6
:10ACF00063463032D258002A14D0012A01D08A4249
:10AD000010DDE164099806900CE03A4600210F201E
:10AD100003F009FE2079A178401C814202D0002076
:10AD200003F017FD618CE08C814229D2BDE6000062
:10AD3000A00000203F420F0038000020A40C00209B
:10AD40003C000020FC0D002082000020A80700200D
:10AD500070000020080500209A9999999999E13F7F
:10AD600000000840A086010000D02724983A000087
:10AD7000600000206400002058000020E70300006D
:10AD80004F4A80188142D1D8A07B0226012800D0EA
:10AD9000A67303F087FB4B4A00210F2003F0C3FD8D
:10ADA000E17800291BD020460A2906D9C5702570F4
:10ADB000FBF77EFBE078002802D0002000F006F9C7
:10ADC000FBF742FAA07C002858D03F490B78637209
:10ADD000487820728A78E271022B16D04EE0A06B80
:10ADE000E16C323881420EDAA1792046491CC9B2A1
:10ADF000A1710229E4D98571069901840670257331
:10AE0000FBF786FFD6E7A571DAE710280ED02F4FA3
:10AE1000062815D0C82831D23818C91CFAF7AEF95F
:10AE200004F016F8642003F0B5F97CE6284F386882
:10AE30004000000E22D1C878FAF782FC38601DE08D
:10AE400021490222C91CB81DFAF7D7F9002815D0EC
:10AE5000207A1D493818E279C91CFAF78FF903F0F6
:10AE6000F7FF7D20F988C000FAF742F919490880F8
:10AE70000146C820FAF73CF917490880002713E07B
:10AE8000114811497D009C388439405B495B8842F8
:10AE900008D02670FBF73CFF002020730A490120F0
:10AEA000B43948537F1CFFB220798742E8D3054A62
:10AEB000002180320F2003F036FD0BB0F0BD000002
:10AEC000983A000000D02724980E00206807002040
:10AED00074000020700000207E000020F8B52F4C88
:10AEE0000546E0692E4A281A411E2062914215D279
:10AEF0000221615E081AFAF72BFC2A4A2A4BFAF75C
:10AF000029FB064608200F46205EFAF721FC324650
:10AF10003B46FAF76DFAFAF751FC208100202070C9
:10AF20001E480423C35E21480288214800888446C5
:10AF3000204806881DE06046484380181E4F80B2B6
:10AF40003880302778436427643078431B4F606132
:10AF5000C01985420BD2C8B219490822088060691D
:10AF6000A25E411BC9188918A161E061F8BD491CA6
:10AF700021702178B142DED3302042431148642150
:10AF80001018484310494118E16160610821401BD5
:10AF9000615EC0184018A061F8BD000028010020C3
:10AFA000CF0700009A9999999999B93FBE0000205E
:10AFB0007E000020700000207C00002078ECFFFF65
:10AFC0007A00002074270000C0BDF0FFFEB5294DB7
:10AFD0002988491C8FB228492F800E88FAF7B8FBC0
:10AFE000264A274BFAF7B6FA0191009025483146D8
:10AFF000FAF77EF8244CE1894218B74206D30020C4
:10B0000028802248019E1018009D02E01046019EF3
:10B01000009DFAF7B1FB33462A46FAF7E9F9FAF749
:10B02000F1FB6081012580B2ED03A84201D3401BF2
:10B030006081E088FAF7A0FB154A164BFAF7F2FA9E
:10B04000064660890F460090FAF796FB32463B466B
:10B05000FAF7CEF9FAF7D6FB80B2A081A84201D365
:10B06000401BA0810C490098096848610098E08164
:10B07000FEBD00007A000020700000201904560E6A
:10B080002D624040E17A0000280100201F050000E9
:10B09000F853E3A59B843E4008050020704700005C
:10B0A000F8B50125124C6D0229462046FCF7CEFB6F
:10B0B00000281BD07D20C00003F06CF829462046F4
:10B0C000FCF7C4FB002811D0EE0005273F072946F6
:10B0D0002046FCF7BBFB0028F9D1642003F05AF8A6
:10B0E000002231463846FCF7B8FBF0E7F8BD000017
:10B0F0000004005010B50448002281898068FCF7E4
:10B10000ACFBFBF7B7FD10BD9026002010B504483E
:10B11000012281898068FCF7A0FBFBF7B1FD10BD1F
:10B1200090260020C3000248C15018188280704742
:10B1300090260020F0B585B04A48FBF7C1FE4A488A
:10B14000FDF77EFA4948FDF787FB4948FDF7C0FD4A
:10B150004848FDF7BDFD4848FDF7BAFD474800786F
:10B16000002801D100F08AFC14216846FAF71FF884
:10B170000024102611270520029469460007019734
:10B1800000960394FCF7A8FAF5010520029469469D
:10B190000007019700950394FCF79EFAFDF722FB48
:10B1A0003748816B020411438163364801680422E9
:10B1B0001143016001210846FCF754FDFDF738FA00
:10B1C00000F0CCFFFFF7E0FA002001F09BFF012028
:10B1D00001F098FF022001F095FF0096012605205E
:10B1E00002946946000701960394FCF775FA05205E
:10B1F000012210210007FCF730FB0520029469466C
:10B200000007019600950394FCF766FA05200122D9
:10B2100029460007FCF721FB1B4D2868C1071BD1FD
:10B220001A4E3168884217D01948017819481429F4
:10B2300001D3FF2101E0FF210902174A01601460D8
:10B24000164A21461460164A0B4614600A460068E6
:10B2500000F0F8FB2868306012A0FEF711FA05B084
:10B26000F0BD0000AC040020D0060020280700201C
:10B2700038050020C00500204806002030000020CE
:10B280000010024000700040280000203400002020
:10B290003800002024000020180000201C0000209E
:10B2A0002000002077616B752075700D0A0000008A
:10B2B000F0B587B003F06AFD5D4800F083FB5D4D9B
:10B2C00028815B48801C00F07DFB68815848001D88
:10B2D00000F078FBA8815948574904464180403422
:10B2E000E18CE1273F01002900D1E78421796970D1
:10B2F00004915248E7844787514AC18E1170514AE0
:10B30000C18F1170504A818F1170A17929704F4AF5
:10B31000817A11704E4986880E604E4A052111804F
:10B32000C0880390F9F7E4FE4B4908800146304697
:10B33000F9F7DEFE8800081886B2484806807D20AE
:10B34000C0007043FAF718FA454A464BFAF76AF913
:10B35000FAF758FA444980B20880009043480680C2
:10B3600043480188C820F9F7C3FE424901220880FA
:10B37000414800260280AF800398E8807D20049930
:10B38000C000002906D12F49E8800A700A21A9804F
:10B390002D490E70E988F9F7ABFE35490880374929
:10B3A0003748009AFCF7BCFB002801D072B6FEE7D4
:10B3B000A08C344D344F012819D134486946088097
:10B3C00072B680213248FBF759FA002804D00222D5
:10B3D00069462F48FBF7F8FA62B62EA002F0BAF8D9
:10B3E000A68403F035FD642002F0D4FEFD60608C7D
:10B3F000012808D111486684068003F029FD6420E5
:10B4000002F0C8FEFD60208C012806D1268403F0DE
:10B410001FFD642002F0BEFEFD600848214A01883D
:10B42000914202D1C088002800D1FD6007B0F0BD74
:10B43000004F0008000000204702000068070020BD
:10B44000B80100207800002079000020660000206C
:10B45000600000206A0000206C00002068000020CE
:10B46000F853E3A59B843E406E000020720000204C
:10B47000700000207E0000207A000020FF7F000086
:10B48000080500200400FA0500ED00E0AAAA00006B
:10B49000384A0008BDF8C8EBC9FDBCB6C4A3CABD94
:10B4A0000D0A0000AA55000000B50449402088623A
:10B4B000FF20F53003F0E8FC00BD00000004005060
:10B4C000FF2302461B0200B519020D489A4202D121
:10B4D00000F0BEF800BD8A4202D100F055F809E044
:10B4E000FF2A04D0824205D100F0FEF800BD00F032
:10B4F00009F800BD002AFCD100F078F800BD00007A
:10B50000FFFFFF0000B500F02FF800F02DF800F06D
:10B510002BF800F029F800F027F800F025F800F0EB
:10B5200023F800F021F800F01FF800F01DF800F0FB
:10B530001BF800F019F800F017F800F015F800F00B
:10B5400013F800F011F800F0B5F800F0B3F800F0CF
:10B55000B1F800F0AFF800F0ADF800F0ABF800F093
:10B56000A9F800F0A7F800BD06484021816100BF9E
:10B5700000BF00BF00BF00BF816200BF00BF00BFAF
:10B58000704700000004005000B500F093F800F090
:10B5900091F800F08FF800F08DF800F08BF800F0D3
:10B5A00089F800F087F800F085F8FFF7DDFFFFF776
:10B5B000DBFFFFF7D9FFFFF7D7FFFFF7D5FFFFF757
:10B5C000D3FFFFF7D1FFFFF7CFFFFFF7CDFFFFF767
:10B5D000CBFFFFF7C9FFFFF7C7FFFFF7C5FFFFF777
:10B5E000C3FFFFF7C1FFFFF7BFFF00BD00B5FFF7C7
:10B5F000BBFFFFF7B9FFFFF7B7FFFFF7B5FFFFF797
:10B60000B3FFFFF7B1FFFFF7AFFFFFF7ADFFFFF7A6
:10B61000ABFFFFF7A9FFFFF7A7FFFFF7A5FFFFF7B6
:10B62000A3FFFFF7A1FFFFF79FFFFFF79DFFFFF7C6
:10B630009BFFFFF799FFFFF797FFFFF795FFFFF7D6
:10B6400093FFFFF791FFFFF78FFFFFF78DFF00BD1F
:10B6500000B5FFF789FFFFF787FFFFF785FFFFF7CB
:10B6600083FFFFF781FFFFF77FFFFFF77DFFFFF706
:10B670007BFF00F01FF800F01DF800F01BF800F051
:10B6800019F800F017F800F015F800F013F800F0C2
:10B6900011F8FFF769FFFFF767FFFFF765FFFFF797
:10B6A00063FFFFF761FFFFF75FFFFFF75DFFFFF746
:10B6B0005BFF00BD0B484021816100BF00BF00BFA0
:10B6C00000BF00BF00BF00BF00BF00BF00BF00BF82
:10B6D00000BF00BF00BF816200BF00BF00BF00BF4E
:10B6E000704700000004005000B5FFF7E3FFFFF7CC
:10B6F000E1FFFFF7DFFFFFF7DDFFFFF7DBFFFFF7FE
:10B70000D9FFFFF7D7FFFFF7D5FFFFF7D3FFFFF70D
:10B71000D1FFFFF7CFFFFFF7CDFFFFF7CBFFFFF71D
:10B72000C9FFFFF7C7FFFFF7C5FFFFF7C3FFFFF72D
:10B73000C1FFFFF7BFFFFFF7BDFFFFF7BBFFFFF73D
:10B74000B9FFFFF7B7FFFFF7B5FF00BD08B5002849
:10B7500008D00246002106480091044B0068FEF71D
:10B7600017F908BD002000F005F808BD75B70008FE
:10B770009C010020044972B60248C860BFF34F8F95
:10B78000704700000400FA0500ED00E0F8B56E4CCB
:10B7900000266E4FE670012038806D49C820088071
:10B7A000A07A401CA072C00706D0E08B411EE18346
:10B7B000022801D2C820E0830120C043FFF706FC25
:10B7C0000A2002F0F0FF7D20400103F007F8614DF0
:10B7D0002020AE7268726048C1887D20C000F9F7F1
:10B7E00087FC68735D4858490078A8732846203163
:10B7F00013380A78027549784175574A1E30917896
:10B800000170D1784170411C10462030027ECA7010
:10B81000407E087150482230027E4A71407E887115
:10B8200000220C39172003F0A9F80021172003F09B
:10B83000B7F8022003F008F8494D01E0FEF70EFCCE
:10B8400000210F2002F01CFF28422063F6D0206B5D
:10B85000411C76D0400472D58122D20100210F20F4
:10B8600003F061F80021102002F00AFF4106394878
:10B87000490E0022B430A16402F052FF354DB435B8
:10B88000687A11285BD102223649681DF9F7B5FCA8
:10B89000002854D1E81F027A69460A70407A48703D
:10B8A000A97A3980C820F9F723FC29492E4F08804E
:10B8B000287BE08328462838C08E388028462838E0
:10B8C000008FA0832948FCF727F96084A08B2849C2
:10B8D000FF30C33080B2A08388420BD94942401860
:10B8E000A08338882249401C80B20B3138808842BE
:10B8F00000D33E8038887D21C9004843A18B401881
:10B900000021206400F0EEF8684600882084A87CBE
:10B9100010492071C731420008460D469130F9F7B1
:10B920002DFC2079294642001248F9F727FCE08BCC
:10B93000FF2804D0267302202070FBF7E9F9F8BD38
:10B94000FFE701F06BFE0000A00000207000002067
:10B950007E000020A40C002068070020B801002011
:10B9600000D027246000002064000020080500208B
:10B97000E7030000140E002070B586B0142168465D
:10B98000F9F715FC0E4E002201213046FBF765FF4A
:10B9900001250024009502946946304601950394E0
:10B9A000FBF79AFE032001900294694600950394E8
:10B9B0003046FBF791FE022002F0ECFB06B070BDB2
:10B9C000000400500088704770470000F8B5044636
:10B9D00000206A461080194D55222A70AA226A70EA
:10B9E0000322AA70661DEE702A716971144A49001B
:10B9F0008918AC712246E81DF9F7C0FB002007E06A
:10BA000029186A468978128889186A461180401C6C
:10BA1000B042F5DB611DA81CFAF7B8FC0146684688
:10BA2000018029190078C87168464078087222465A
:10BA300009320249002001F003FCF8BDCC0B0020C4
:10BA400068070020F8B5164604460F460122052077
:10BA50001D46D1030007FBF700FFFFF725FD204639
:10BA6000FFF72EFD3846FFF72BFD3046FFF728FD88
:10BA70002846FFF725FDFFF717FDF8BD10B501219A
:10BA800005200022C9030007FBF7E7FE10BD0000F8
:10BA9000FFB505468400114881B01E4620180422D7
:10BAA0000A9FF9F76BFB0D4804222C3020180399EC
:10BAB000F9F764FB09480949583020180660680006
:10BAC000B0314018397801707978417004480349E1
:10BAD000006D8431085105B0F0BD0000000F00205A
:10BAE000A0000020FEB50D46FFF7F8F92448FCF74A
:10BAF00013F8244C80B2208201900A20401BC00021
:10BB0000F9F726FE06460F46A069F9F735FE1E4AEC
:10BB10001E4BF9F787FD00900D460198F9F72CFEB2
:10BB20002B46009AF9F764FC32463B46F9F760FC75
:10BB3000F9F768FE85B26581E088F9F71DFE124AC3
:10BB4000124BF9F76FFD06460F462846F9F714FE2B
:10BB500032463B46F9F74CFCF9F754FE81B201201E
:10BB6000C003A181814201D3091AA181854201D379
:10BB7000281A60810249608909684861E081FEBD38
:10BB80000805002028010020F853E3A59B843E40CF
:10BB900010B5FAF713FBFDF719FE00280DD0FDF7DD
:10BBA00015FE0B24E40100190069002805D0FDF7FB
:10BBB0000DFE0019016902A08847002010BD000099
:10BBC0004F4B0D0A0000000010B5FAF715FBFDF70A
:10BBD000FDFD00280DD0FDF7F9FD0B24E40100194F
:10BBE0000069002805D0FDF7F1FD0019016902A0E8
:10BBF0008847002010BD00004F4B0D0A00000000D8
:10BC000010B5022814DAFDF7E1FD00280DD0FDF78C
:10BC1000DDFD0B24E40100190069002805D0FDF7C3
:10BC2000D5FD0019016907A088470020C04310BD59
:10BC30004868F9F7EFFA002801D1FDF72BFC002046
:10BC400010BD000064656275675F6F666620666C94
:10BC500061670D0A0000000010B5022814DAFDF734
:10BC6000B5FD00280DD0FDF7B1FD0B24E40100194E
:10BC70000069002805D0FDF7A9FD0019016907A09A
:10BC800088470020C04310BD4868F9F7C3FA002870
:10BC900001D1FDF705FC002010BD00006465627550
:10BCA000675F6F6E20666C61670D0A0010B5FFF765
:10BCB00021FAFDF78BFD00280DD0FDF787FD0B2441
:10BCC000E40100190069002805D0FDF77FFD001987
:10BCD000016902A08847002010BD00004F4B0D0AEB
:10BCE0000000000010B5FFF711FAFDF76FFD002806
:10BCF0000DD0FDF76BFD0B24E4010019006900284D
:10BD000005D0FDF763FD0019016902A088470020F6
:10BD100010BD00004F4B0D0A0000000070B5FDF78C
:10BD200055FD0B25ED0100280CD0FDF74FFD401906
:10BD30000069002806D0FDF749FD401902690FA1EE
:10BD400011A09047FDF742FD002815D0FDF73EFDFC
:10BD50004019006900280FD0FAF7D0F9F9F770FD03
:10BD600004460E46FDF732FD401905690B48224690
:10BD7000017833460AA0A847002070BD76312E30E6
:10BD80002E302E340000000056657273696F6E3AD3
:10BD900020202020202025730D0A000038000020DC
:10BDA000426174746572793A202020202020257524
:10BDB000252520252E3266560D0A000010B51121CA
:10BDC0000248FDF7CDFC002010BD0000E0EE0008A9
:10BDD0000020704710B5072814D0FDF7F7FC0028A5
:10BDE0000DD0FDF7F3FC0B24E401001900690028D5
:10BDF00005D0FDF7EBFC0019016903A0884700207E
:10BE0000C04310BD002010BD75736167653A207294
:10BE100074635F7365742079797979206D6D20641E
:10BE200064206868206D6D2073730D0A00000000A7
:10BE300010B50020FFF78AFC002010BD10B50B24C0
:10BE4000E401062812DAFDF7C1FC00280BD0FDF74B
:10BE5000BDFC00190069002805D0FDF7B7FC0019EA
:10BE600001690BA088470020C04310BDFDF7AEFC60
:10BE700000280BD0FDF7AAFC00190069002805D0A6
:10BE8000FDF7A4FC0019016911A08847002010BD2E
:10BE90007365745F616463206E6F726D616C5F6D5A
:10BEA000696E206E6F726D616C5F6D617820657276
:10BEB000726F725F6D696E206572726F725F6D6115
:10BEC00078206572726F725F636E740D0A000000F5
:10BED0004F4B0D0A0000000010B50B24E4010228AE
:10BEE0000FDAFDF773FC00281BD0FDF76FFC00197B
:10BEF0000069002815D0FDF769FC001901690AA046
:10BF00000EE0FDF763FC00280BD0FDF75FFC001985
:10BF10000069002805D0FDF759FC0019016904A04B
:10BF20008847002010BD00004552524F520D0A00B4
:10BF30004F4B0D0A0000000070B500250B24ED43A7
:10BF4000E40102280FDAFDF741FC002822D0FDF7BA
:10BF50003DFC0019006900281CD0FDF737FC0019D2
:10BF6000016916A015E04868F9F754F9002801D0D6
:10BF7000082811D9FDF72AFC00280BD0FDF726FC74
:10BF800000190069002805D0FDF720FC001901699F
:10BF90000EA08847284670BDFDF718FC00280BD07E
:10BFA000FDF714FC00190069002805D0FDF70EFC10
:10BFB0000019016908A08847002070BD7365745F8F
:10BFC0006465765F69642069640D0A0069642065B0
:10BFD00072726F720D0A00004F4B0D0A00000000D4
:10BFE00010B50B24E401032812DAFDF7EFFB00285B
:10BFF0000BD0FDF7EBFB00190069002805D0FDF719
:10C00000E5FB001901690BA088470020C04310BD63
:10C01000FDF7DCFB00280BD0FDF7D8FB0019006909
:10C02000002805D0FDF7D2FB001901690AA0884756
:10C03000002010BD7365745F6970205B7365727654
:10C0400065725F69705D205B7365727665725F70A3
:10C050006F72745D0D0A00004F4B0D0A0000000066
:10C0600010B50B24E401032812DAFDF7AFFB00281A
:10C070000BD0FDF7ABFB00190069002805D0FDF7D8
:10C08000A5FB001901690BA088470020C04310BD23
:10C09000FDF79CFB00280BD0FDF798FB0019006909
:10C0A000002805D0FDF792FB001901690AA0884716
:10C0B000002010BD7365745F77696669205B7373D8
:10C0C00069645D205B70617373776F72645D205B80
:10C0D00069705D0D0A0000004F4B0D0A0000000062
:10C0E00010B5FFF727F8002010BD10B5FEF718FABD
:10C0F000002010BD034A1168382389B299430143D7
:10C10000116070470030014070B5104C2078002855
:10C1100011D00025012806D002280FD0032801D114
:10C12000FEF70CFC70BDFFF731FB607B411C6173B7
:10C1300009E0257070BDFAF7BBF970BDFAF7E8FDAC
:10C14000207B411C21730528F3D870BDA00000207E
:10C1500010B5FDF749FCFBF79BFB10BD10B59AB07D
:10C1600034216846F9F723F8142115A8F9F71FF8C8
:10C1700020210DA8F9F71BF8224801680324E402E6
:10C18000A143C21489180160FBF764FD1E480169D0
:10C19000A143016106200090FF20013002900120A0
:10C1A0000390102004900220099040040B9000019D
:10C1B00000240C900A946846FBF7C0FF002801D0C9
:10C1C00072B6FEE70F20159003201690179418946E
:10C1D0000121199415A8FBF743FE002801D072B67F
:10C1E000FEE787200D9003200F9480041490109494
:10C1F00011940DA8FBF76AFD002801D072B6FEE786
:10C200001AB010BD007000404010024002490148C1
:10C21000886070470050000800ED00E0F0B402684C
:10C220000124A407144D154E154FA04205D0A84275
:10C2300003D0B04201D0B84203D170239A434B6877
:10C240001A43A04205D0A84203D0B04201D0B84260
:10C2500004D103231B029A43CB681A4380239A43D9
:10C260000B691A4302608A68C2620968816201210F
:10C270004161F0BC7047000000040040000801402C
:10C280000014014010B4C906C90E01238B40046A92
:10C290009C430462036A8A401343036210BC7047E4
:10C2A00030B48468FF252D02AC431B0213430B43BB
:10C2B0002343836030BC7047826870239A430A43EB
:10C2C00007210A438260704730B4026A5208520064
:10C2D0000262026A446883697025AB439B089B0035
:10C2E0000D681D4302239A438B68134344608561A4
:10C2F00049684163036230BC704730B4026A10235E
:10C300009A430262036A4568826907242403A243B0
:10C3100003242402A2430C682402144320229343E2
:10C320008A6812011A434560846149688163026228
:10C3300030BC704730B4026AFF2301339A43026273
:10C34000026A4468C3697025AB439D08AD000B6861
:10C350002B4301256D02AA438D682D0215434460CD
:10C36000C3614968C163056230BC704730B4026A7A
:10C3700001231B039A430262036A4568C2690724CA
:10C380002403A24303242402A2430C68240214437E
:10C390000122520393438A6812031A434560C46121
:10C3A00049680164026230BC704730B4036A046AB1
:10C3B0006408640004628469F025AC4312012243DE
:10C3C0000A24A3430B438261036230BC704730B43C
:10C3D000036A1024A34303628369046A0F252D03B3
:10C3E000AB4312031A43A0239C43090121438261FA
:10C3F000016230BC7047000070B5FF24114D01345C
:10C40000AC62AF20800001F0CCFEAC6102F066F9B6
:10C410000D4C0E4DA06007E002F060F9A060FDF742
:10C420001DFE6068401C6060A068A842F4D102F064
:10C4300039F800206060FFF767FE02F033F802F081
:10C4400019F870BD00040050800000203001CADEE1
:10C4500010B509480949806A88420BD3642001F06D
:10C4600099FEBFF34F8F07490548C860BFF34F8F50
:10C4700000BFFDE710BD00000000002000943577EC
:10C480000400FA0500ED00E010B4818CC90707D064
:10C4900001684A6801235B049A43836A1A434A602D
:10C4A000818C890707D501684A6801231B049A43D8
:10C4B000C36A1A434A60818C490707D501684A68F4
:10C4C00001239B049A43036B1A434A60818C09073A
:10C4D00007D501684A680123DB039A43436B1A437B
:10C4E0004A60818CC90607D501688A6801231B034D
:10C4F0009A43836B1A438A60818C890607D5016849
:10C500008A6801235B039A43C36B1A438A60818C58
:10C51000490612D501684B6801221205046C934349
:10C5200023434B60016C914207D101684A680323A1
:10C530005B059A43436C1A434A60818C090607D510
:10C5400001684A680123DB04806C9A4302434A6015
:10C5500010BC7047F0B583B00446264600278036ED
:10C560007760FBF781F90290206800682546000794
:10C57000603500281CDA2A48009001210022490574
:10C580002046029B00F09AFC002811D0EFF31081A6
:10C59000012080F310882068026880239A4302609B
:10C5A00081F310882020E0672F76032003B0F0BDD0
:10C5B00020680068400729D5194800900121002211
:10C5C00089052046029B00F079FC00281ED0EFF37D
:10C5D0001081012080F3108820680268FF23213336
:10C5E0009A43026081F31088EFF31081012080F3F9
:10C5F00010882068826852085200826081F3108897
:10C60000202030602F76032003B0F0BD2020E067AB
:10C610003060276667662F76002003B0F0BD00000B
:10C62000FFFFFF0110B5806A0022014640314A83B6
:10C630004A82FCF76FFB10BDF8B5846AE06F2546AF
:10C6400080352E682168896800270906002906DAE6
:10C65000212804D152200753204600F0DFF820683B
:10C660008068400606D5222E04D15A200753204662
:10C6700000F090F868681021084368602046FCF7D5
:10C6800049FBF8BD70B50146886A0968096800234E
:10C690008906002937DB5A210B52EFF31082012162
:10C6A00081F3108801680C68FF250135AC430C60EC
:10C6B00082F31088EFF31082012181F31088016862
:10C6C0008C68640864008C6082F31088EFF3108239
:10C6D000012181F3108801688C684025AC438C608F
:10C6E00082F31088202280210A50016E01290AD18C
:10C6F000EFF3108281F3108801680C681025AC43B9
:10C700000C6082F310884366016E012902D0FCF7A9
:10C71000A7FD70BD5821095AFCF7D8FA70BD10B5B5
:10C72000806A01214166016E012902D0FCF79CFD5F
:10C7300010BD5821095A4908FCF7C8FA10BD10B5B8
:10C740000146886A0968096889061BD400225221BB
:10C750000A52EFF31082012181F3108801688B687F
:10C760008024A3438B6082F31088EFF310810122B1
:10C7700082F310880068026840231A43026081F344
:10C78000108810BDFCF780FE10BD10B5806AFCF764
:10C790007FFE10BD10B4EFF31082012181F31088E9
:10C7A00001680B68FF242134A3430B6082F31088D7
:10C7B000EFF31082012181F3108801688B685B0818
:10C7C0005B008B6082F31088016E01290AD1EFF3C0
:10C7D000108281F3108801680B681024A3430B605A
:10C7E00082F31088202280210A5000210166816690
:10C7F00010BC704710B5EFF31082012181F310884F
:10C8000001680B684024A3430B6082F31088202149
:10C81000C1670021C166FCF737FE10BD10B4EFF30D
:10C820001082012181F3108801680B68C024A343A2
:10C830000B6082F310882021C16710BC7047000094
:10C8400070B5014640318B8B024680321568144624
:10C850000268222D04D0906908210843906170BDC0
:10C86000526A456D1A402A80426D921C42654A8B7D
:10C87000521E4A834A8B002AF1D1EFF31083012222
:10C8800082F3108802681568FF262136B5431560CB
:10C8900083F31088EFF31083012282F3108802687B
:10C8A00095686D086D00956083F3108820222260E2
:10C8B000002484664466184B02689A420ED053687E
:10C8C0001B020BD5EFF31083012585F31088156843
:10C8D0000126B606B543156083F31088026E012A5F
:10C8E00002D0FCF7BDFC70BD0466EFF3108301229B
:10C8F00082F31088026815681024A543156083F33D
:10C9000010880268D369DB43DB0600D41462098B0C
:10C91000FCF7DCF970BD00000048004070B501462E
:10C9200040318B8B02468032156814460268222DF6
:10C9300004D0906908210843906170BD526A1A4082
:10C94000436D1A70426D521C42654A8B521E4A83D7
:10C950004A8B002AF1D1EFF31083012282F3108871
:10C9600002681568FF262136B543156083F31088E9
:10C97000EFF31083012282F31088026895686D0836
:10C980006D00956083F31088202222600024846665
:10C990004466184B02689A420ED053681B020BD5AE
:10C9A000EFF31083012585F3108815680126B6067C
:10C9B000B543156083F31088026E012A02D0FCF79C
:10C9C0004FFC70BD0466EFF31083012282F31088E0
:10C9D000026815681024A543156083F31088026867
:10C9E000D369DB43DB0600D41462098BFCF76EF9D4
:10C9F00070BD000000480040F8B504460025904F87
:10CA000020682269A168E369114362691A431143EE
:10CA100002688C4B1A400A43026020684168032276
:10CA200012039143E26811434160A0692168B94251
:10CA300001D0226A10438A680B231B029A430243E7
:10CA40008A608149226881488A4213D1C068800780
:10CA5000800F07D0012809D0022805D0032807D06D
:10CA6000102142E0012140E002213EE004213CE0AF
:10CA700008213AE076498A4213D1C0680C21084067
:10CA800007D0042809D0082805D00C2807D0102189
:10CA90002BE0002129E0022127E0042125E00821E4
:10CAA00023E06C498A4201D100211EE06A498A4292
:10CAB00001D1002119E0BA4216D1C06803218902D0
:10CAC00008400BD001218902401A0BD0401A07D030
:10CAD000884201D1082108E0102106E0002104E08D
:10CAE000022102E0042100E010215D485B4E83003A
:10CAF000BA4236D1002913D0022914D0042917D004
:10CB0000082918D000200125002861D06268510052
:10CB10005118814202D8110381420FD2012589E0C8
:10CB2000FBF7A2FAF0E73168C906EDD41846EBE747
:10CB3000FBF7BAFAE8E70120C003E5E7010E0602B9
:10CB40005008002330185941F8F7E8FA0321090288
:10CB5000444A411A914202D82168C8606AE001251E
:10CB600068E00122E769D203974234D1092919D23A
:10CB70000F007F443F79FF19BF4404070A140F14C4
:10CB800014141200FBF770FA0EE0FBF77DFA0BE0CD
:10CB90003168C90608D4184606E0FBF785FA03E0B9
:10CBA000104601E000200125002843D061684000C4
:10CBB0004A088018F8F79CFA02462B49103A8A4234
:10CBC00007D8491C01400007420F0A432068C26091
:10CBD00030E001252EE0092919D20F007F443F796A
:10CBE000FF19BF4404070A140F1414141200FBF7B2
:10CBF0003BFA0EE0FBF748FA0BE03168C90608D4AF
:10CC0000184606E0FBF750FA03E0104601E000206A
:10CC1000012500280ED061684A081018F8F768FA54
:10CC20000146114A1039914203D8216880B2C86088
:10CC300000E001250020A066E0662846F8BD00005F
:10CC400000480040F369FFEF003801404010024007
:10CC500000440040004C00400050004000100240E2
:10CC600000093D00FFFC0F00EFFF000070B5044617
:10CC700061655820025300212546803569602220D5
:10CC80002860606F002819D0214BC362636F214870
:10CC90001863636F20485863606F81632168666D15
:10CCA000134624313246606FFAF78DFB002805D019
:10CCB0001020686020202860012070BD20690028B5
:10CCC0000CD0EFF31081012080F3108820680268F7
:10CCD000FF2301331A43026081F31088EFF31081C0
:10CCE000012080F310882068836801221343836049
:10CCF00081F31088EFF3108182F310882068826836
:10CD000040231A43826081F31088002070BD000028
:10CD100085C600081FC7000839C6000870B4416501
:10CD2000014640310A834A830024846601238268D5
:10CD30001B03FF259A4207D10269002A01D08D8387
:10CD400019E02B4A8A8316E07F26002A09D00125A4
:10CD50002D07AA420ED10269002A09D03F228A83F8
:10CD600009E00269002A01D08E8304E08D8302E08D
:10CD70008E8300E08C83014680314C6022220A6061
:10CD8000EFF31082012181F3108801688C6801257E
:10CD90002C438C6082F310888168994202D101692A
:10CDA000002912D0134981660169002910D0EFF3E0
:10CDB0001081012282F3108800680268FF2321336A
:10CDC0001A43026081F310880EE00B498166EBE79D
:10CDD000EFF31081012282F310880068026820239B
:10CDE0001A43026081F3108870BC00207047000075
:10CDF000FF0100001DC9000841C8000810B4C16F40
:10CE0000212910D1014640314A8A002A0DD0C26C36
:10CE100003681288D205D20D9A62C26C921CC26459
:10CE2000488A401E488210BC7047EFF310820121EF
:10CE300081F3108801680B688024A3430B6082F3A0
:10CE40001088EFF31081012282F3108800680268D5
:10CE500040231A43026081F3108810BC704710B45D
:10CE6000C16F21290ED1014640314A8A002A0BD0D8
:10CE7000C26C036812789A62C26C521CC264488AFF
:10CE8000401E488210BC7047EFF31082012181F3ED
:10CE9000108801680B688024A3430B6082F310881C
:10CEA000EFF31081012282F31088006802684023AA
:10CEB0001A43026081F3108810BC7047FFB583B03D
:10CEC0000C9D04460E4617462068C16930468843CB
:10CED00027D00020B84245D120468030029020382B
:10CEE0000190681C36D0FAF7BFFC0699401AA84298
:10CEF00019D8002D17D02068016849072AD5C169C3
:10CF0000C943090712D42068082505622046FFF7A7
:10CF100041FC02984560019900200876012007B085
:10CF2000F0BD0120D6E7032007B0F0BDC069C043C3
:10CF300000050FD401202168C00208622046FFF7D7
:10CF400029FC0298202141600199002008760320E5
:10CF500007B0F0BD2068C1693046884305D0002085
:10CF6000B842BED0002007B0F0BD0120F8E70000B5
:10CF700010B50248FBF7D2FE10BD0000C00500202E
:10CF800010B50248FBF7CAFE10BD0000480600209D
:10CF9000F8B51D4D0E0034D0032832D27421484319
:10CFA0001A494418A078002802D0012822D028E08D
:10CFB000E168A068421860680090406F00684068AF
:10CFC0002769101A0818C01BF8F792F8012905D82C
:10CFD00017D100980068C069800612D43878307084
:10CFE00061692069884201D1A06800E0401C20618D
:10CFF000002506E0204618303146FCF797FA002855
:10D00000F6D02846F8BD0000FFFFFFFFB82C002037
:10D0100070B50C00064601D0032E02D30020C04399
:10D0200070BD7421484321490E54227845186A7016
:10D030006078A8706068A860A168E9606278002ADA
:10D0400002D0012A05D00BE028614018401E68611B
:10D0500006E0284618300123A2686168FCF741FA0F
:10D06000E068E86220692863A069286760696863EE
:10D070002078002801D0012806D121460C310EC9A4
:10D0800028463830FCF7BFFE6078002804D001281D
:10D0900006D0022804D006E0304600F009F802E08D
:10D0A000304600F021F8002070BD0000B82C0020B0
:10D0B00038B50C497422504342185068016804E0A6
:10D0C0004C6A6B461C801C881C80CB691B07F7D4FC
:10D0D00091681161D368CC18641E54619AB2FCF750
:10D0E00057F838BDB82C002074214843044910B5C6
:10D0F00040180146683140680122FCF77DF810BDF8
:10D10000B82C002070B5054674201A4968434418AD
:10D11000A078002802D0012807D00DE0A068206187
:10D12000E1684018401E606106E020461830012387
:10D13000E268A168FCF7D5F96078002801D00128E1
:10D1400006D121462C310EC920463830FCF75BFE53
:10D15000A078002804D0012806D0022804D006E0D8
:10D160002846FFF7A5FF02E02846FFF7BDFF002095
:10D1700070BD0000B82C002070B50D0001D0032850
:10D1800002D30020C04370BD7421484304494418B1
:10D1900074212046FCF758FC0020656070BD00003B
:10D1A000B82C002010B502460E49002074234343DA
:10D1B0005B185B6893420FD17422424351188978FF
:10D1C000002906D0012901D0022901D1FFF78CFFE7
:10D1D00010BDFFF76DFF10BD401CC0B20328E5D3A2
:10D1E00010BD0000B82C002038B5014613480024BB
:10D1F00074226243121852688A4219D17421614321
:10D200000818817801290BD0022908D1016F002963
:10D2100002D0806EC0B288472046FFF765FF38BD58
:10D22000816E6A46117069461830FCF73FF9F3E7E2
:10D23000641CE4B2032CDBD338BD0000B82C002002
:10D24000F7B582B00021009103991546002903D05B
:10D25000002D01D0032803D30020C04305B0F0BD4A
:10D26000742148432B4946187078344638340028D6
:10D2700004D0012820D0022842D049E0FCF73AFA35
:10D2800020462946FCF791FD070033D02046394659
:10D29000FCF757FD2A4638680399F7F76FFF2046D9
:10D2A000FCF765FD0446FCF7B3FBA088216882B259
:10D2B0007068FCF74BF82BE0FCF71CFA2046294677
:10D2C000FCF773FD070015D020463946FCF739FD01
:10D2D0002A4638680399F7F751FF2046FCF747FDC7
:10D2E0000446FCF795FBA088216882B27068FCF7C1
:10D2F00087F80DE0FCF78CFB0020C043009007E0AE
:10D30000134664204343AAB270680399FBF7ADFF4C
:10D310000098A3E7B82C002070B51F4A00217423A1
:10D320004B439B185B68834231D1742041438C1876
:10D330006078002816D0012813D1204638300546E1
:10D34000FCF715FD01462846FCF7E5FC2846FCF7EE
:10D350000EFD002805D081888AB201686068FCF75C
:10D360004FF870BD204638300546FCF700FD0146F9
:10D370002846FCF7D0FC2846FCF7F9FC0028F0D042
:10D3800081888AB201686068FBF7E0FF70BD491CC4
:10D39000C9B20329C3D370BDB82C0020F8B53E4CE8
:10D3A000002321783D4A1D46082910D0072947D07F
:10D3B000062950D0052952D0042953D0032954D02E
:10D3C000002956D0012958D002295AD05BE0A17813
:10D3D00000264A1F04E0314FBF5DFB189BB2761C4C
:10D3E0009642F8DB667927799A195118E3786278C2
:10D3F000C9188918C9194018C0430006000E1AD16F
:10D40000012E14D0022E16D125482449C018F7F752
:10D41000B5FE01F01DFD642000F0BCFEBFF34F8F90
:10D4200021492048C860BFF34F8F00BFFDE759086E
:10D430001046FEF7CBFA2570E570A570A571F8BD12
:10D44000A1795054491CC8B2A071A178491F8842E3
:10D45000F5D1082001E0607007202070F8BDE07071
:10D460000620FAE760710520F7E7A070E570042058
:10D47000F3E7552807D10120EFE7AA2803D10220BE
:10D48000EBE7032803D02570E570A570F8BD0320F5
:10D4900020702071F8BD000097000020680B00206C
:10D4A000680700200400FA0500ED00E070B5174C95
:10D4B000206B002828D12169A06A401A0A2823D3AA
:10D4C0000025656228462562FF23E5610246014684
:10D4D000A361FEF7B7FAFEF78FFFA06A2061E0892B
:10D4E0000B4A401C80B2E0811178032901D3E58109
:10D4F00006E0052804D9032902D20120A07000E02B
:10D50000A5701570FEF7BAFA70BD0000000000208B
:10D51000AB00002070B50D48FAF7FEFA0C4C01255F
:10D520002082AD0309E00948FAF7F6FA80B22082BA
:10D53000A189FF392D39884206DBA18980B2884252
:10D54000F1D349198842EED870BD000008050020CB
:10D55000280100200FB410B503A9044B044A029817
:10D5600000F00CFA10BC08BC04B01847EDE9000844
:10D57000A40400207CB51546024600201C46002964
:10D580000BD0491E00920191044B6A462146284661
:10D5900000F0F4F9009A002111707CBDB5E000089C
:10D5A0002021020C01D010211046020A01D01046A1
:10D5B0000839020901D01046091F820801D010461F
:10D5C000891E420801D0881E7047081A7047F0B4BF
:10D5D000040C8BB2264682B25E430D0C1046370C0B
:10D5E0005843360480190021794116466E43370CA2
:10D5F00036048019794126466E438919F0BC70477C
:10D6000030B47446641E2578641CAB4200D21D46BB
:10D61000635D5B00E31830BC18470000BFF34F8F19
:10D6200004490348C860BFF34F8F00BFFDE7000007
:10D630000400FA0500ED00E0BFF34F8F04490348F2
:10D64000C860BFF34F8F00BFFDE700000400FA057C
:10D6500000ED00E000487047A804002002E008C880
:10D66000121F08C1002AFAD170477047002001E05C
:10D6700001C1121F002AFBD1704708B5002168467E
:10D6800001706B46012202212C2001F05BF902217E
:10D69000684601706B4601222C2001F053F908BD49
:10D6A00038B504466D20694608706B46012207496B
:10D6B0002E2001F047F90649002C01D0054A00E070
:10D6C000054A2E2001F024F938BD000006080000AC
:10D6D00006180000070600000716000038B50446CB
:10D6E0006B4602220021362000F0FEFFB32123000A
:10D6F000FFF786FF0E0F08153A3A3A3A1C273A3AD6
:10D700002F34483A002168460170407841084900AA
:10D7100014E06946087880088000401C04E06946EF
:10D72000087880088000801C08701DE06846027838
:10D730000A404832027041788020014368464170B7
:10D7400012E0684602780A40027040784106490EAD
:10D75000F4E7694648780221084303E069464878BF
:10D76000FD210840694648706B46012200213620A1
:10D7700001F0E8F8012200AB11463620013301F038
:10D78000E1F838BD69460878CF2108406946203065
:10D79000CAE708B5032168464170012101706B4654
:10D7A00002220021362001F0CDF80122D203062109
:10D7B0002D2001F0ADF8012000F0ECFC0120FFF776
:10D7C0008DFF08BD08B5020A69464A7008706B46AD
:10D7D000022204212D2001F0B5F8032069460870CB
:10D7E0006B46012206212D2001F0ACF8002069468D
:10D7F00008706B46012206212D2001F0A3F80A21B2
:10D800002D2000F03DFF08BDF0B51FB486B009988B
:10D81000089A030D0021024314D05148514A1818A8
:10D82000504305141198012810981AD0281A401C4A
:10D8300000264D4F4D49009601910490002812DAC0
:10D84000444211E01198012449A3012801D1109804
:10D85000C1430698119A84600360C26041600BB0B6
:10D86000F0BD4042E4E70446210500203F4A001C89
:10D8700051410391029012E0E00707D032463B4647
:10D8800001990098F7F766FE0191009032463B46F9
:10D8900010461946F7F75EFE06460F466410002C48
:10D8A000EAD10498039B0028029A0999089806DA9D
:10D8B000F7F750FE019B009AF7F74CFE05E0F7F7EB
:10D8C000B1FE019B009AF7F7ADFE04460E4600221A
:10D8D000284BF7F7DDFF03D80020C043014607E0DF
:10D8E0000022254B20463146F7F782FDF8F70CF968
:10D8F000102409E0002C0ADB0A220023F7F70EFCB3
:10D90000079B30321A55641E02460A43F2D1112297
:10D91000641C079B121B1C19119B012B03D00123B4
:10D9200008430ED10AE0084304D0112010900020D3
:10D93000119077E71098151A6D1E0BE0109882422F
:10D9400002DD00236D1C03E0824201DA00236D1E1C
:10D95000002BEED0069811998260C16030C07EE73E
:10D9600001FCFFFF104D0000000014400000F03FDC
:10D97000300000000000F0430000E03FFFB597B02A
:10D980000646002518E2252877D100242746FD49C0
:10D99000049400E00443761C32780120203A904041
:10D9A0000842F7D130782A280ED00222307801467A
:10D9B0003039092916D804990A23594330394018B7
:10D9C0001443761C0490F1E7189802C8049118904B
:10D9D000002904DA01204003044348420490022055
:10D9E0000443761C30782E2814D104200443707828
:10D9F000761C2A2809D11898761C80C8189009E04E
:10DA00000A214F43303FC719761C30780146303920
:10DA10000929F5D930786C2810D006DC4C281AD0AA
:10DA200068280ED06A2817D104E0742813D07A2809
:10DA300012D110E00120400504430CE0012109054A
:10DA400001E0032109050C437178814203D10120D3
:10DA500000052418761C761C3078119066280BD0AF
:10DA600013DC58287DD009DC00287BD04528F6D06F
:10DA70004628F4D047281AD1A5E118E0632835D00C
:10DA8000642870D0652812D19DE170286CD008DC24
:10DA90006728F1D069287BD06E280DD06F2806D179
:10DAA000BAE073282ED0752871D0782859D01A9AE8
:10DAB000199990476D1C7EE16002400F022809D041
:10DAC00003280DD00428189801680DD00D60001DA2
:10DAD000189070E11898EA1701680D604A60F6E73F
:10DAE000189801680D80F2E70D70F0E718986A4603
:10DAF00001781172001D18900020507202A8009049
:10DB0000012005E0189802C8189000200091C04339
:10DB100061070DD5002101E00199491C0191B9422D
:10DB200012DA8142F8DB009A515C0029F4D10BE053
:10DB3000002101E00199491C01918142FADB019A1F
:10DB40000099895C0029F5D1019904981A9B471A1C
:10DB500021463846199A00F097FA0199401945185C
:10DB60000BE04FE02CE113E04EE0009800990078C4
:10DB7000491C00911A9A199990470198401E0190EA
:10DB8000401CF2D1214638461A9B199A10E137E021
:10DB90000A200021009001916002410F022907D064
:10DBA000189A01CA1892C2179446032908D00AE0AD
:10DBB0001898C01DC108C90005C91891944607E00E
:10DBC00000B2C2179446042902D140B2C1178C4654
:10DBD00000226146944506DA0A46002140429141FE
:10DBE0008C462D2102E0210504D52B216A461173B4
:10DBF000012103E0E10701D02021F7E7029155E080
:10DC00000A200AE0102008E01020009000210420E3
:10DC100004430191082703E00820002101910090AE
:10DC20006002410F022907D0189A01CA18920022F7
:10DC30009446032908D008E01898C01DC108C900FF
:10DC400005C91891944603E080B2042900D1C0B2FE
:10DC500000210291210729D51199702906D0009A37
:10DC60001021019B4A401A4305D00EE040216A462C
:10DC70001173012108E06146014306D030216A4654
:10DC800011731199517302210291009A0821019B8D
:10DC90004A401A430AD16146014301D1610705D5C3
:10DCA00030216A46117301217F1E02911199582972
:10DCB00004D035A10E910DA90D910DE037A1F9E722
:10DCC0006146019B009AF7F729FA0E9B8C469B5CF4
:10DCD0000D9A521E0D92137061460143F0D10D98BA
:10DCE00005A9081A20300190600703D5012000041F
:10DCF000844300E001270198874201DD381A00E0E3
:10DD00000020019900904118029809180498401ABF
:10DD10000490E00306D421461A9B199A049800F057
:10DD2000B3F94519002706E003A81A9AC05D1999AE
:10DD300090476D1C7F1C02988742F5DBE0030CD5F1
:10DD400021461A9B199A049800F09EF9451904E09F
:10DD50001A9A3020199990476D1C0099481E00901E
:10DD60000029F5DC08E00D980D990078491C0D910B
:10DD70001A9A199990476D1C0199481E0190002923
:10DD8000F1DC63E1092801003031323334353637B4
:10DD900038396162636465660000000030313233F7
:10DDA0003435363738394142434445460000000097
:10DDB00000F05AF94519761C3078002800D0E2E5C9
:10DDC00028461BB0F0BD600700D406271898C01D78
:10DDD000C108C90048680A680831C30FDB071891F9
:10DDE000190001D09CA108E0210501D59BA104E008
:10DDF000E10701D09AA100E09AA1430011985B08C5
:10DE0000109165280CD006DC452809D046281DD085
:10DE1000472841D141E0662818D067283CD13CE032
:10DE20000021112F01DB112000E0781C01910090EE
:10DE300008A911A8FFF7E8FC139905910021119A90
:10DE400015927F1C12980197009150E00120C007A5
:10DE500003900120019008A9009711A8FFF7D4FCB6
:10DE6000139A149905920022119B0092129815930F
:10DE7000059A0192002901D0104602E0791C401851
:10DE80000190381A01D5019804E04042401E0090EC
:10DE9000781C0190C01B029043E0012F00DA01279B
:10DEA0000021112F01DD112000E038460191009082
:10DEB00008A911A8FFF7A8FC13990591119A002150
:10DEC000129815920091019721070CD40599B94237
:10DED00001DB019900E00191012904DD159A491E39
:10DEE000515C302906D0B84201DA011D05DA012162
:10DEF000029115E00199491EEDE7002805DC009923
:10DF0000411800910199091A03E0019A411C9142BC
:10DF100000DD01910099401A401C02900120C007C9
:10DF20000390200706D402990198814202DB002069
:10DF3000C043029000206946C87707AF01210398CB
:10DF40000337C907884224D0022011902B20129059
:10DF5000039800280CDA404203902D20129007E02D
:10DF60000A210398F7F7C4F830317F1E0390397007
:10DF70001199481E11900029F2DC03980028EFD176
:10DF8000791E129808703078202108404530BF1E55
:10DF9000387006A8C01BC01D039010980078002898
:10DFA00000D00120019941180298C0170918039860
:10DFB00009180498401A401E0490E00306D4214634
:10DFC0001A9B199A049800F05FF845191098007888
:10DFD000002803D01A9A199990476D1CE00324D5A4
:10DFE00021461A9B199A049800F04EF845191CE036
:10DFF0000098002807DB00990598884203DD1598F2
:10E00000405C199901E0199930201A9A90470098BC
:10E010006D1C401C00900298401E0290002804D104
:10E020001A9A2E20199990476D1C0199481E01904B
:10E030000029DDDC05E038781A9A7F1C1999904791
:10E040006D1C0399481E03900029F4DC21461A9B9D
:10E05000199A0498ACE600002D0000002B00000087
:10E060002000000000000000F8B5044600251E4610
:10E070001746880404D405E039462020B0476D1CBB
:10E08000641EF9D52846F8BDFFB50446002581B0C9
:10E090001E46C80301D5302700E02027880404D598
:10E0A00005E038460399B0476D1C641EF9D5284633
:10E0B00005B0F0BD4A68002A06D00A68531C0B6000
:10E0C00010704868401E486070470000F8B54A006C
:10E0D0002B4B520DD6182B4A0C460546142E2BDA24
:10E0E000002E12DA284BF7F783F900221346F7F7D0
:10E0F000CFFB40D2002C03DA0124E40700253AE0EC
:10E100002046284337D0214C14E0214F0B46F740DE
:10E110003B402B4331D01C4BF7F76AF900221346E2
:10E12000F7F7B6FB27D2002C03DD01200005F040F5
:10E130000419BC4300251EE0332E1EDC33460027A5
:10E14000143BFF43DF40384217D00F4BF7F7FAF983
:10E1500000221346F7F79CFB0DD2002C0ADD142E8B
:10E160000CD03420811B012088404019A84200D2E5
:10E17000641C0546BD4321462846F8BD641CF9E7EA
:10E1800001FCFFFF9C7500883CE4377E0000F03FF7
:10E19000FFFF0F007D2110B5C900484300F001F8D2
:10E1A00010BD002140E000BF00BF00BF00BF00BFA6
:10E1B00000BF00BF00BF00BF00BF00BF00BF00BF67
:10E1C00000BF00BF00BF00BF00BF00BF00BF00BF57
:10E1D00000BF00BF00BF00BF00BF00BF00BF00BF47
:10E1E00000BF00BF00BF00BF00BF00BF00BF00BF37
:10E1F00000BF00BF00BF00BF00BF00BF00BF00BF27
:10E2000000BF00BF00BF00BF00BF00BF00BF00BF16
:10E2100000BF00BF00BF00BF00BF00BF00BF00BF06
:10E2200000BF00BF00BF491C8142BCD37047000043
:10E23000FEB504460020064601906079764940000C
:10E240000F5A617875482578491E6A460163117036
:10E25000042D7CD0072D7AD0002102912178017302
:10E260006E49E379012292058969002B71D09143AF
:10E2700081616A48217A4173217A82698907890B11
:10E280000A4382610021042000F04DFB3A466449B4
:10E290002E2000F03DFB68460078FFF701FA614F41
:10E2A0000522785D810040185F49431807212B2023
:10E2B00000F048FB5D49029801220B180B21282031
:10E2C00000F040FB785D5A4980000A580C21282054
:10E2D00000F029FBE079574980004018A1794900F6
:10E2E000425A0221272000F013FB68460078524969
:10E2F00040000A5A0421272000F00AFBE079002898
:10E300002BD0A07804282ED028206946087220221D
:10E310000621272000F0FCFA02AB0122262127204B
:10E3200000F010FB68460078444900014018E1788D
:10E33000890042580821272000F0F5FAA17A601CD4
:10E34000627A0902114313D016E000E001E00121D6
:10E3500083E71143FF0881618BE7642206212720B0
:10E3600000F0D6FADEE71020694608720246CFE7D1
:10E3700033490172090A4172417A007A0A02024362
:10E380002021272000F0C4FA2E4F0C2123203A68C8
:10E3900000F0C9FA6846007804214000C01982885C
:10E3A000232000F0B5FAA07900280AD0E0792649A8
:10E3B000012243180021212000F0C4FA0320012685
:10E3C00001902A07120F1001024360780021800794
:10E3D000000B0243019800050243700402432079B8
:10E3E000C006400902436079C00602431F2000F0C6
:10E3F0009AFAA07861780123084302040748DB03F6
:10E400000261E179490319430A43026100210820AE
:10E4100000F089FA0020FEBDC0EF0008142E002095
:10E420000428000068EF0008C4010020E201002079
:10E4300070EF000890EF00089CEF0008A0EF0008C4
:10E440004110000088EF0008E401002038B50C46B8
:10E4500007498A8B002102432C2000F059FA6846B4
:10E4600004706B46012206212C2000F06BFA38BDA7
:10E47000142E002010B5FFF700F910BD10B50446AA
:10E480000421362000F0FCF80121C902002C01D043
:10E49000084300E0884302460421362000F043FA96
:10E4A00010BD000038B540206946087000210E20DC
:10E4B00000F0E6F80446002211460E2000F033FA80
:10E4C0006B46012200210D2000F03CFA074A002192
:10E4D0000F2000F028FA00F001FA224600210E2059
:10E4E00000F021FA02480021017338BDF8FF27240B
:10E4F000342E0020FEB50546042069460870514CB4
:10E500000020607521462031206348710873A08384
:10E510006063A06300F0E2F84B4E206002E000F080
:10E52000DDF82060B042FAD10020FFF7D7F800F004
:10E53000D5F8464E20603078242801D9243806E0EA
:10E540000621F6F7D5FD0622101A400108430206FF
:10E5500001040A4301020A430243B26070600021D1
:10E560001E2000F0E0F900F0B9F820606B460122AF
:10E570000021242000F0E6F91E20FFF723F986B2DF
:10E58000300AA0730420FFF71DF9074600F0A6F833
:10E5900020603806000E0DD002206946087101ABDC
:10E5A000012212212D2000F0CDF9A08B01210903B9
:10E5B0000843A08300F092F820600620FFF702F9DC
:10E5C00060600720FFF7FEF8A060F006C00E20751F
:10E5D00001D110202075C0B200F0F0F9E80707D093
:10E5E000FFF7D7F8A08B0121C9020843A0830AE0F6
:10E5F0000521362000F02EF8154908400246052175
:10E60000362000F085F90120FFF768F8002104208A
:10E6100000F036F8A0610021262000F031F8152125
:10E620008903084302460021262000F07CF90022DD
:10E630002621362000F06CF900F050F82060002010
:10E64000FEBD0000142E00203001CADEB8010020FB
:10E65000FFFD000038B5094C89B280B26B4602223A
:10E6600000F042F8002806D168464078010268466A
:10E670000078081884B2204638BD0000FFFF000073
:10E6800038B50024E44389B280B26B46042200F01E
:10E690002BF8002806D103216846435C2202D418D7
:10E6A000491EFAD5204638BD38B500246B460322F2
:10E6B0002821272000F018F8022069460B5C22026E
:10E6C000D418401EFAD5E00202D50348204338BDD5
:10E6D000E002C00A38BD00000000F0FF10B50021C4
:10E6E0000846FFF7CDFF10BD38B5002909D04024FA
:10E6F00020436C462070C8B27F2906D86070022083
:10E700000AE069460870012006E0802420436C4638
:10E710006070C809A0700320694600F071FB38BD25
:10E7200010B5144603460A4621461120FFF7DCFFC8
:10E7300010BD10B50346052200211520FFF7D4FFB8
:10E7400010BD10B50346052200211720FFF7CCFFAE
:10E7500010BD38B5054600206946087000F0BEF8C7
:10E76000FF2401342246002D01D003221202002191
:10E770000D2000F0CDF8002D13D06B4601220321AF
:10E780000F20FFF7B1FF68460078000709D5FFF7B3
:10E7900089FE224600210D2000F0BAF80020C04377
:10E7A00038BD002038BD10B5044600211A20FFF7FF
:10E7B00067FF000D22030005120B024300211A20FF
:10E7C00000F0B1F810BD000010B5024602492E203D
:10E7D00000F09EF810BD000004180000F8B50546D2
:10E7E0006B46012203210420FFF77EFF0126114C16
:10E7F0003607002D0DD02A4600210C2000F088F8A5
:10E80000694608781021084369460870A0693043BA
:10E8100007E069460878EF21084069460870A0695A
:10E82000B0430B46A06101220321042000F08AF8C6
:10E83000F8BD0000142E002010B50246002118205B
:10E8400000F066F810BD0000F8B5074600256846E0
:10E850000570B807204C2E4600280ADA8020694649
:10E8600008706B46012200210D2000F06BF801209A
:10E870002073F8076946087821D0062108436946C5
:10E8800008706B46012200210D2000F05BF8032187
:10E890000F20FFF7DFFE8121C900084219D0402078
:10E8A000694608706B46012200210D2000F04AF8ED
:10E8B0000020FFF7E3FD00252673ED4309E0022168
:10E8C0000843694608706B46012200210D2000F0C4
:10E8D00039F82846F8BD0000342E00201CB56B46E0
:10E8E000012203210F20FFF7FFFE68460078402237
:10E8F000C1091040C9014000814208D00120694689
:10E900000871024601AB03210D2000F01BF81CBD6D
:10E9100008B56B461A70120A5A7089B280B2022288
:10E9200000F010F808BD38B500236C46E254120A16
:10E930005B1C042BFADB89B280B22346042200F070
:10E9400001F838BD38B58024002909D0C0252843F6
:10E950006D462870C8B27F2907D86870022009E088
:10E96000204369460870012004E020436870C8090C
:10E97000A8700320694600F08DFA38BD10B5144622
:10E98000012312189B029A4202D90020C04310BDF5
:10E990000B46821E21460920FFF7D4FF002010BD40
:10E9A00010B5054A8905126901430A430021082070
:10E9B000FFF7B9FF002010BD142E002038B5044623
:10E9C0006B4601220E212B20FFF78EFE6846007851
:10E9D000E10640094001C90E0143684601706B46DB
:10E9E00001220E212B20FFF7ADFF38BD38B50446BC
:10E9F0006846047069460320ABBE204638BD7CB52E
:10EA0000002425466846FFF794FE04206946220E3E
:10EA10002D02154322020C5C1443401EF7D52046FC
:10EA200029467CBD7CB5002425466846FFF789FE53
:10EA300004206946220E2D02154322020C5C144369
:10EA4000401EF7D5204629467CBD000070B51A4D02
:10EA50001A4C2868E168401A0A282BD9A0780028A7
:10EA600028D00120E070164801781648FBF78CFD8D
:10EA70002868E060A079FF21401CA0711248134A69
:10EA8000002501601560124A28461560114A0346A8
:10EA900015600246FCF7D6FF6420F8F7CDFCFCF7C2
:10EAA000EDFFA0790A2802D9E570A570A5710AA02A
:10EAB000FAF7E6FD70BD00002800002038000020B5
:10EAC0005A01002078160020200000202400002099
:10EAD0001C000020180000206C6F726120627566B7
:10EAE000610D0A00F8F7DCFEFDF738FBFBF7B6FD19
:10EAF000FBF77CFDFBF756FEFBF7E6FEFBF700FF9E
:10EB0000FBF76CFEFBF790FE2748264901600021C9
:10EB1000416081600162254A416242618162F8F789
:10EB20008BFF002801D072B6FEE7FCF7C1FBF7F7B8
:10EB300061FEF7F72FFEFF2007214130FFF786FC2B
:10EB4000FFF798FCF7F752FAF7F76EF9FCF796FF24
:10EB5000FCF7D0FAFF20000203461A461146FCF7E4
:10EB600071FFFF24F5342046F8F766FCFF2000040F
:10EB700003461A461146FCF765FF2046F8F75CFC91
:10EB800000231A4619461846FCF75CFF2046F8F7A2
:10EB900053FCF7F771F9FEF789FCF7F7E1FAFDF797
:10EBA00057FCF6E7007C004008050020FFFF00004E
:10EBB00010B50446FBF7EAF94E20FBF7B9F9FBF76D
:10EBC00021FAE0B2FBF7B4F9FBF71CFAFBF7DEF928
:10EBD0004F20FBF7ADF9FBF715FA0020FBF77AF9A8
:10EBE0000446FBF7EFF9204610BD70B50D4604460C
:10EBF000FBF7CCF94E20FBF79BF9FBF703FAE0B2E9
:10EC0000FBF796F9FBF7FEF92846FBF791F9FBF7BE
:10EC1000F9F9FBF7D7F90A20FFF7C3FA70BD000036
:10EC200010B52421002000F04DF81B48FFF7B9FA79
:10EC300000210F2000F046F80521102000F042F8D6
:10EC40000421112000F03EF883217F2000F03AF8E3
:10EC500069217F2000F036F8BD217F2000F032F8D6
:10EC60000E480078262804D1002240218C2000F094
:10EC700019F8012000F02AF80948142101872820FA
:10EC800000F020F80A20FFF78CFA012000F036F897
:10EC9000012000F043F810BD204E0000A00100202C
:10ECA00068070020F8B517460E4605460024FFF712
:10ECB0007FFF3946B44331402143284600F002F833
:10ECC0000020F8BD10B5FFF790FF10BD10B500286B
:10ECD0000AD000212720FFF7F5FF04211920FFF7B4
:10ECE000F1FF8721162005E000211620FFF7EAFF3B
:10ECF00000211920FFF7E6FF10BD000010B5002825
:10ED000001D0002200E0802280211120FFF7CAFFFD
:10ED10000148FFF746FA10BDA086010010B5002893
:10ED200011D001212F20FFF7CDFF62213020FFF706
:10ED3000C9FF46213120FFF7C5FF32210846FFF702
:10ED4000C1FFA22100E022213320FFF7BBFF10BD4D
:10ED50000C480D4A0188914210D1C18832290DD347
:10ED6000C18E43290AD8818F012907D8C08F012875
:10ED700004D8044840308088012801D90120704718
:10ED80000020704768070020AA55000010B5012236
:10ED9000920217491748F7F78BFD15481649028864
:10EDA0008A4223D0018015498180FF21F531C1803D
:10EDB0000A2101810021418181810122C281818357
:10EDC0004323C38602230387E1231B0143878287F2
:10EDD000C28702464032118451849184C18391805C
:10EDE000142484821182D38400F032F810BD000014
:10EDF0006807002000FC0008AA550000341200003B
:10EE0000F0B58C460025FF260F4901368E620F4C67
:10EE100008E067467F5DE760A768FF07FCD0E7680A
:10EE20001F706D1C8542F4DB0020074606E0E7609A
:10EE3000A568ED07FCD0E5681D54401C9042F6D350
:10EE40008E610020F0BD0000000400500030014041
:10EE500070B5FFF77DFF002801D0012070BD72B6AC
:10EE60000124074DA40221462846F7F707FD002894
:10EE700004D0224603492846F7F7A6FD62B670BDC6
:10EE800000FC000868070020002100E0491C8142C6
:10EE9000FCD37047F0B50025FF260F4F9C46013686
:10EEA0000B46BE620D4C06E0595DE160A168C907E2
:10EEB000FCD0E1686D1C8542F6DB002007E061466E
:10EEC000095CE160A168C907FCD0E168401C904280
:10EED000F5D3BE610020F0BD0004005000300140B9
:10EEE00034F10008EBC000081CF1000831BE000836
:10EEF000F4F000081DBD0008D8F0000859BC000857
:10EF0000ACF0000801BC00080CF10008D1BD0008FD
:10EF100014F10008D5BD000898F000083DBE0008B7
:10EF200004F10008E1BF0008A0F0000839BF0008A4
:10EF3000CCF0000861C0000824F10008D9BE000828
:10EF4000ECF00008E5BC0008C4F00008ADBC000807
:10EF5000E4F00008C9BB0008B8F0000891BB000845
:10EF6000FCF00008E1C000080000010203040005F5
:10EF7000405C0000A05C0400C06C0800805C0400E1
:10EF8000E03F1E00E07D1E0007A9022570889B88D7
:10EF90000A001600010006000100020087008D0033
:10EFA0002D001A3152001A339A001A351D011A37F2
:10EFB0006B003B31BE003B335E013B3596023B3775
:10EFC000000099599959EB518F421E45142E00802B
:10EFD000EB51F5283333E13A703DE13AC235852BE8
:10EFE000C2353333C235C235AE47E13A5138A3306A
:10EFF0005138000000000000000001020304060771
:10F000000809030406080C10182030000000000155
:10F0100002030400404040404040404040414141E4
:10F0200041414040404040404040404040404040DE
:10F0300040404040050202020202020202020202B5
:10F040000202020220202020202020202020020274
:10F0500002020202029090909090901010101010F6
:10F0600010101010101010101010101010101002AE
:10F07000020202020288888888888808080808082E
:10F080000808080808080808080808080808080206
:10F090000202024014F000087365745F616463004B
:10F0A0007365745F6465765F6964000064656275AA
:10F0B000675F6F6666000000626565705F6F666619
:10F0C000000000006770735F6F6666007365745FB1
:10F0D000776966690000000064656275675F6F6E3E
:10F0E00000000000626565705F6F6E006770735F9F
:10F0F0006F6E0000696E666F00000000736C6565DE
:10F10000700000007365745F697000007274635F63
:10F11000676574007274635F736574007265626F13
:10F120006F7400007365745F636F6E7472617374E3
:10F130000000000074657374000000002B2B2B0D81
:10F140000000000061742B6A6F696E3D6F7461612D
:10F150002C31300D0000000061742B63683D636E3C
:10F160003437302C330D000061742B64723D350D43
:10F170000000000061742B6170706575693D353267
:10F1800036393733363936653637343834360D004C
:10F1900061742B636C6173733D610D0061742B614D
:10F1A00070706B65793D3262376531353136323892
:10F1B00061656432613661626637313538383039BD
:10F1C0006366346633630D0061742B6D6F64653D57
:10F1D0006D61630D0000000061742B6164723D6F0E
:10F1E00066660D0061742B7265626F6F740D0000AE
:10F1F00061742B736C6565703D6C696768742C3045
:10F200002C6C6576656C2C6C6F770D0061742B64CB
:10F2100065766575693D3437333635343966303057
:10F220003331253034780D00636C65617200000065
:10F230006C73000054F2000800000020AC040000D1
:10F24000385C0008E4F20008AC040020BC30000088
:10F250006CD60008014B4350011204125002368054
:10F260001405021415090901026281395001890748
:10F270002452030CE5800CC9B88933133CF11B08F8
:10F28000C8041A44041A9004130CF21B0874081AD8
:10F290009C041A68041A58041AD8041AF0041AE4D0
:10F2A0000441022327130704380D091E08054008EE
:10F2B0002609104008560A131D043B08BE053ED817
:10F2C000BC40100894920402212032021A28A01394
:10F2D00025971B0830081AD90801FF01FF0176B2F3
:04F2E0000100000029
:04000005080050C1DE
:00000001FF
